:020000040100F9
:1000000038480020E5000001ED000001EF0000018C
:1000100000000000000000000000000000000000E0
:10002000000000000000000000000000F1000001DE
:100030000000000000000000F3000001F5000001D6
:10004000F7000001F7000001F7000001F7000001D0
:10005000F7000001F7000001F7000001F7000001C0
:10006000F7000001F7000001F7000001F7000001B0
:10007000F7000001F7000001F7000001F7000001A0
:10008000F7000001F7000001F7000001F700000190
:10009000F7000001F7000001F7000001F700000180
:1000A000F7000001F7000001F7000001F700000170
:1000B000F7000001F7000001F7000001F700000160
:1000C0000348854600F056F80048004751050001F6
:1000D0003848002040BA7047C0BA70470138FDD197
:1000E000704700000448804704480047FEE7FEE7E9
:1000F000FEE7FEE7FEE7FEE795030001C100000111
:1001000030B50B46014600202022012409E00D46AF
:10011000D5409D4205D31D469540491B2546954037
:1001200040191546521E002DF1DC30BD03460B432D
:100130009B0703D009E008C9121F08C0042AFAD29D
:1001400003E00B780370401C491C521EF9D2704723
:10015000D2B201E00270401C491EFBD2704700225F
:10016000F6E710B513460A4604461946FFF7F0FFB6
:10017000204610BD064C0125064E05E0E36807CC7D
:100180002B430C3C98471034B442F7D3FFF79CFF45
:10019000C0070001D0070001F7B5D4B004460E46F1
:1001A00000205390052052900025002700BFEFF358
:1001B00010800090FF21453101A8FFF7D0FF00F02B
:1001C000F1F905462448854218D1012000038442F4
:1001D00002D1002053902AE001204003844202D142
:1001E0004011539023E003200003844203D10120F7
:1001F000400253901BE0529857B0F0BD174885421B
:1002000013D101200003844201D153900FE001205B
:100210004003844201D1539009E00320000384424B
:1002200001D1539003E05298E6E75298E4E705AF16
:100230000137FF2241320A4901A8FFF777FF012069
:1002400000F04FF93146569A5398B84752900098AB
:1002500000F047F95298CFE7C440130085601300BF
:10026000E8050001F1B58AB0002009907D20C000AA
:1002700008900125AD020027002007907F200690FE
:1002800040240026002005900390200102900020C9
:1002900001903E490A98884206D83D4800686102AC
:1002A00088433B49086006E0394800680121C903DA
:1002B0000843374908607D21C9000A98FFF720FFED
:1002C0007D21C9000090FFF71BFF450100BF3048AA
:1002D00000687F21090288430190200201990843A8
:1002E0002B4908600520FFF7F9FE10E00120FFF719
:1002F000F5FE2748406B02210840002800D007E0A7
:100300000598411C05910899884200D900E0EDE765
:1003100000BF1F48C06B86B2AE4201D9771B00E018
:10032000AF1B0298874203D2E0B20390B8B20290AA
:10033000AE4201D3069400E007940699079840184E
:10034000C005000E04900498A04200D103E0049C74
:1003500009988742BBD800BF0D4800687F21090279
:1003600088430190039800020199084308490860F6
:100370000846406840084000486000BF04484068A4
:10038000042108400028F9D10BB0F0BD0090D00343
:100390000010024010B53E48C0690121090708431A
:1003A0003B49C861812000063A4908633A484861E0
:1003B0003A4808623A48006803218903884338496B
:1003C00008603421374800F073F836480069401C53
:1003D000002803D033480069002817D12C48406812
:1003E0000121090408432A4948600846406807215A
:1003F00009028843264948600846406809150843B1
:10040000234948602848FFF72DFF3FE021488069D5
:100410004409640123480078C006C00E04431D4807
:1004200084611B4800680121C9038843184908609A
:10043000084600687F21090288430446194800697C
:10044000000220431249086008464068012109045F
:1004500008430F494860084640680721090288435D
:100460000B49486008464068091508430849486038
:100470000846006A0D490840054908620846006AB6
:100480000849C968090208430149086210BD000013
:1004900000100240007000400F0800001800020029
:1004A00000100140004000200090D003FF00F8FF42
:1004B00070B504460D462A46214601200003FFF789
:1004C0006BFE70BD02E008C8121F08C1002AFAD1F5
:1004D00070477047002001E001C1121F002AFBD1C4
:1004E000704780F31088704730B502460B460021F4
:1004F000C94312E01078521C414000240BE0480828
:10050000CD07ED0F002D01D0074D00E0002568401C
:100510000146601CC4B2082CF1DB18465B1E0028A3
:10052000E8D1C84330BD00002083B8ED0446012067
:10053000C007204305490863206880F3088800BF8E
:1005400062B66068804700BFFEE7000000700040B0
:10055000114C124D1249206888421AD12821204698
:10056000FFF7C2FFA16A884213D16168022902D154
:100570002146183101E0214608310846074A016842
:10058000914205D32122D2040168914200D205682C
:1005900000BF2846FFF7CAFF0040000100800001AD
:1005A00011C011CA70B5D2B00024002500BFEFF30E
:1005B00010800646FF21453101A8FFF7D0FD01ACB0
:1005C00001349822074901A8FFF7B0FD0120FFF789
:1005D00088FFA04705463046FFF783FF284652B004
:1005E00070BD00002807000140BA7047C0BA7047CC
:1005F0000138FDD170470000F7B50325AD06286A24
:1006000082B016460C46400840002862286A022143
:1006100008432862286A8007FCD4662068600127A6
:100620002F61A86AC005FCD5992068602F61A86A6F
:10063000C005FCD5FF209130FFF7DAFFFF2301331F
:10064000AB626846EF60352169602F61A96AC90510
:10065000FCD5AB62A969EF60C9B205226A602F615F
:10066000AA6AD205FCD5AB62AA690902D2B21143CB
:100670000180C80702D0032005B0F0BDAB626869F5
:10068000FF210831884368616869C91E08436861B1
:1006900002980002483068600820A860EE602F6170
:1006A000A86AC005FCD5FF200130A8620023F61C13
:1006B000B0080ED0B2081148006899006054060ACC
:1006C00009194E70060C000E8E705B1CC8709A42A1
:1006D000F1D8FF200130A8626869FF210831884302
:1006E0006861686938436861286A80088000286208
:1006F000286A38432862002005B0F0BD8000000C55
:10070000032080064169FF2208329143416142691A
:1007100001210A434261026A920892000262026A5F
:100720000A43026270470000002003218906096A1B
:10073000490849000322920611621146096A022201
:10074000114303229206116200BF03218906096A40
:10075000022211400229F8D0D101032292069162AF
:100760000321D1609F2151600121116100BF03214C
:100770008906896AFF22013211409142F7D1032292
:1007800092069162114688694969FF2208329143B5
:100790000322920651611146496901221143032245
:1007A000920651611146096A890889001162114651
:1007B000096A012211430322920611627047000068
:1007C000D00700010040002038080000D4040001D8
:1040000011C011CA010000000080000150CF000063
:1040100054BC3C60000000000000000000000000F4
:0C40200000000000000000005ABD8DDD13
:10800000C8B70020698100017181000169AD0001DC
:108010000000000000000000000000000000000060
:108020000000000000000000000000002DB1000171
:1080300000000000000000002781000131B10001B4
:108040007B8100017B8100017B8100017B8100013C
:108050007B8100017B8100017B8100017B8100012C
:108060007B8100017B8100017B8100017B8100011C
:108070007B8100017B8100017B8100017B8100010C
:108080007B8100017B8100017B8100017B810001FC
:108090007B8100017B8100017B8100017B810001EC
:1080A0007B8100017B8100017B8100017B810001DC
:1080B00039B300017B8100017B8100017B810001DC
:1080C0000348854601F076F80048004785F5000131
:1080D000C8B7002040BA7047C0BA70470138FDD118
:1080E0007047000040BA7047C0BA7047704670478A
:1080F000084B19680868203080F30988022080F353
:108100001488BFF36F8F3FBCAE4608BC04BC62B698
:1081100018470000A4470020EFF3108072B67047A4
:1081200080F310887047EFF309800E4B1A682038EF
:108130001060F0C044464D4656465F46F0C008B554
:1081400072B60AF0AFFD62B60CBC11680868103058
:10815000F0C8A046A946B246BB4680F3098820383D
:10816000F0C81847A4470020044880470448004747
:10817000FEE7FEE7FEE7FEE7FEE7FEE789B1000166
:10818000C180000130B50B460146002020220124A9
:1081900009E00D46D5409D4205D31D469540491B3B
:1081A0002546954040191546521E002DF1DC30BD84
:1081B00070B500242546002801DA01244042002938
:1081C00001DA01254942FFF7DDFFAC4200D0404211
:1081D000002C00D0494270BDF0B51FB40646002007
:1081E00082B005464024019100901BE0019922468F
:1081F0000F46304600F02DFE049A059B801A9941E7
:1082000010D310461946224600F013FE361A8F414D
:108210000197224601200021009F00F00AFE381835
:108220004D4100902046641E0028DFDC019B009831
:108230002946324607B0F0BD01464139192900D818
:10824000203070470549064A08685043054A80189F
:10825000086040087047014908607047FC470020EB
:108260006D4EC6413930000003460B439B0703D0D7
:1082700009E008C9121F08C0042AFAD203E00B78EB
:108280000370401C491C521EF9D27047D2B201E063
:108290000270401C491EFBD270470022F6E710B561
:1082A00013460A4604461946FFF7F0FF204610BD64
:1082B000421C0178401C0029FBD1801A704710B580
:1082C000002200E0521C835C8C5CA34201D1002B95
:1082D000F8D1D8B2E1B2401A10BDC9B203E00378B8
:1082E0008B4203D0401C521EF9D20020704730B59B
:1082F00004460020034600E05B1C934203D2E05C8E
:10830000CD5C401BF8D030BD03460A780270401C9B
:10831000491C002AF9D11846704730B5054600209F
:10832000034600E05B1C934205D2EC5CC85C201A5B
:1083300001D1002CF6D130BD0FB400B58DB009903D
:108340000B9010A900200091C0430A9000200C90CF
:1083500006480690064807906A4609A80F9900F05B
:10836000B1FD0DB008BC04B018470000E58E000157
:10837000058F0001FFB5087889B01546FF2805D0A4
:10838000491C2D2804D00022002407E000240BE023
:108390000122F9E70A235C430419491C0878FF28E5
:1083A000F8D1002A00D06442002004902A780146C7
:1083B0002D2A01D02B2A0FD16D1C2D2A02D000228C
:1083C000049209E00122FBE700260A2233466D1CD5
:1083D00000F0F2FC381871412F78FF2FF4D10C9A7D
:1083E000A218069202460A4304D0FF23069A91334C
:1083F000DA4205DA002109980A4606C00DB0F0BD40
:108400000024B74AB54D2646079200F011FC0290B1
:1084100006980391002801DA474200E00746390533
:108420000020AF4A001C51410191009012E0F80772
:1084300007D022462B463046079900F0D9FA064667
:10844000079122462B461046194600F0D1FA044601
:108450000D467F10002FEAD10698019B0028009A54
:108460000399029806DA00F02BFB3246079B00F0D6
:1084700027FB05E000F0BCFA3246079B00F0B8FA93
:10848000049A002A02D00122D2075140099A03C25D
:10849000B4E7FFB591B0002009900025ED432E20F0
:1084A0009E685C681F460190B9696D1C12988847E8
:1084B0000090396A88470028F6D10098401C0AD0FD
:1084C0000D20C0018443002E12DD00982B2809D016
:1084D0002D280DD103E00020C04315B0F0BD0120D0
:1084E00080020443B9696D1C12988847761E00907B
:1084F00003A9600501D52D2000E02B206A461073EA
:10850000491C0CA80F9102900AE0B9696D1C1298E1
:10851000884700900120400204431398761E0560AE
:10852000002E02DD00983028EFD001990098884293
:1085300046D18020044308E00998401E099001209C
:10854000400204431399681C0860B9696D1C761ECB
:108550001298884700903028EED031E00199884287
:1085600005D1200603D480200443761E1EE0009827
:1085700003F0F0F8002826D001204002044307A9A8
:108580000F980331761E88420BD200980F9930382D
:1085900008700F98401C0F90200607D50998401EC0
:1085A00003E0200602D40998401C0990A00502D5DA
:1085B0001399681C0860B9696D1C1298884700906F
:1085C000002ECBDC59E0002E57DD0098652801D045
:1085D000452852D1A00550D5032000028443B96933
:1085E0006D1C761E129888470090002E0CDD2B28FB
:1085F00004D02D2808D1FF2001300443B9696D1C37
:1086000012988847761E0090E00501D52D2100E0E4
:108610002B21029801700298401C0290019025E0E5
:108620000120400204430EA902980131761E8842BF
:108630000ED20098029930380006000E087003D15F
:108640000299019881420AD90298401C029006E0E2
:10865000E00501D5234801E0224840420990B9696C
:108660006D1C12988847009013980560002E04DD59
:10867000009803F06FF80028D2D1F9691298884762
:108680000F99FF200870029903AA087000200A9031
:108690000B900CA90AA8099BFFF76CFEA00502D459
:1086A0000120C04319E72420044209D0E00713D178
:1086B00038680B9A0A99031D3B60006806C00BE0FE
:1086C0000B990A9800F05CFB0146E00704D138687A
:1086D000021D3A60006801602846FEE60000144072
:1086E0000000F03FF1D8FFFFF7B582B00F4600263B
:1086F000029C02F01BFF0090006801902578641C2A
:10870000002D05D000F0CAFB0068405DC007F5D120
:108710002B2D02D02D2D1CD0641E0098002101604D
:1087200039462046049A00F0FFFB0146002F04D092
:108730003868A04201D10298386000980068022889
:108740000BD00098019A0260700506D5484205B02A
:10875000F0BD012080020643DFE70846F7E7F8B5E1
:1087600002464A40D40F42004B0052085B089A422E
:1087700002D20246084611464A0023D0C30D4A00E1
:10878000DDB2120EAD1A202D35DA49020126490A52
:10879000F6058A19002C00D0524220214F1B1146A9
:1087A000B9402A411018C20D9A4221D0002C17D08E
:1087B000012D08DCDA05801AD20F8019D207DBB24E
:1087C00000F060FCF8BDDA05801A012340001B06AA
:1087D000C01880185A428018CA0F1043490007E099
:1087E0004908C2071143DA05801A80194008801829
:1087F00000F040FCF8BD61000122511A001BF7E7B0
:108800000122D2075140AAE70122D2075040A6E731
:10881000024670B54A40D30FDB0740002DD04A0016
:108820002AD0010E140E000212020919400A520A3F
:108830008418E50104465443000A120A2E045043EA
:10884000A4194219200CC543AA18120C0125AD0326
:10885000521C521912047F39240400D0521C1043B8
:1088600001D44000491EC2B20C06C0092018401CA9
:108870004008802A02D003E0002070BD400840007C
:10888000002900DA0020184370BD0000F0B507464B
:108890000846584087B0C00F049048000E46590063
:1088A00040084908BC1A884105D2384631461E4660
:1088B00017460B4602465800400810434CD0300D76
:1088C000039040055900400D490D0590401A029053
:1088D000402872DA18030121000B090508430190B2
:1088E00004980092002805D0019952420020884146
:1088F00000920190029840210A1A0199009800F014
:1089000098FA05460C466B4607CB00F0B3FAC0193F
:108910007141039A0E0D0023D71756401A467A402C
:10892000164344D0049A002A2DD0029A012A039AB1
:1089300015DC1205C01A914101263605001C714153
:10894000D20F059ED2070093019202962A46234633
:1089500000F0DEFB07B0F0BD38463146FAE71605F9
:10896000224A0F46B218C01AB74101210905001C5E
:108970004F4100187F41114618187941E20F10430A
:108980006D19644113E0E2076D0815436408C207DE
:108990001443039A01261205C01A91413605001CA2
:1089A0007141CE07400830434908C01851412A465A
:1089B000234600F0A0FBCDE7FFE70498012240002A
:1089C000C117121A00238B4104983146C417381A74
:1089D000A141EEE730B40124E407634030BC55E721
:1089E00030B40124E407614030BC4FE70000E0FFF1
:1089F000F0B51FB488B00B99099800244840099934
:108A0000C00F490049080991C0070B99009049001F
:108A100049080B9109990898A64608431CD00B9960
:108A20000A98084318D0099801244000420D4800D4
:108A3000410D099824050003000B204309900B9871
:108A40000003000B20430B9050181C4940180022D3
:108A500001901446104605E0002001460DB0F0BD1F
:108A6000032801DA034600E003239C46C11A0AAE3C
:108A70000AE05F0008ADED5B4F00F75B7D43002728
:108A8000AA187C41491C5B1E6145F2DD410004AB24
:108A90005A522104120C0A43240C401C0828DFDB24
:108AA000019802900099704601910090059B049AEC
:108AB0000799069800F02CFBD0E700000DFCFFFFA3
:108AC000F0B50C465C4085B0E40FE40703944C001D
:108AD000002664085900944649080246029622433B
:108AE00021D062460A431ED06200570D4A000E0391
:108AF0002303550D012402462C492405781B1B0B2A
:108B0000360B401823432643614600901C46501AFA
:108B1000B44103D30098401C009002E092180098E2
:108B20005B41002803DA0020014605B0F0BD0020BB
:108B3000012109050746864611E064461D46141BBF
:108B4000B54106D36546521BB341744607430C43F7
:108B5000A646CD0740084908284392185B410546C0
:108B60000D43EAD11046184313D0604619465040D1
:108B70007140084306D06046101AB34106D2012264
:108B8000002306E000220123DB0702E00122D2439A
:108B90005310009874460105381C6141029C039DE6
:108BA0000019694100F0A7FABFE70000FD030000CB
:108BB00070B54B005B0803430BD04B005C0D0026E7
:108BC00033466542B341D417AD1AA34102DB0020FE
:108BD000014670BD12053018514170BD10B500221C
:108BE0009623114600F04EFA10BD00000EB5C217D4
:108BF000C10F5040CA0740180021054B0293019253
:108C000000910A460B4600F083FA03B000BD000055
:108C1000330400000EB505490291002100910A4677
:108C20000B46019100F074FA03B000BD330400005C
:108C30000EB5054A0292002200921346019200F0FE
:108C400067FA03B000BD000033040000C20F41000A
:108C500040020123400ADB05D207090EC0187F2914
:108C600001DA00207047962903DC9623591AC84080
:108C700001E096398840002AF4D040427047000055
:108C800070B5CD0F4A0009030123090B1B051943D9
:108C90000B4BED070024520D9A4201DA002070BD03
:108CA000074B34339A4203DC9A1A00F0D2F802E000
:108CB0000449511888402C43F1D0404270BD000057
:108CC000FF030000CDFBFFFF4A0009030123090B4E
:108CD0001B0519430A4B10B5520D9A4202DA0020C7
:108CE000014610BD064B34339A4203DC9A1A00F059
:108CF000B0F810BD034BD21800F09BF810BD000077
:108D0000FF030000CDFBFFFFC20FD2074000400869
:108D10000BD0C10D0723DB01C91840020905400A29
:108D20001143C208400711437047002001467047B5
:108D300010B5002904DB0124E40740428C412146A0
:108D4000002B04DB1C460123DB075242A3418B426C
:108D500000D1824210BD000010B5002904DB0124BF
:108D6000E40740428C412146002B04DB1C460123D2
:108D7000DB075242A341994200D1904210BD00004E
:108D8000CB0FDB07490010B5490802460A4307D05C
:108D90000A0D07240903E401090B121B002A01DC58
:108DA000002010BDC900440F0C43C100E018D205DB
:108DB000801800F05FF910BDF0B51FB486B0002038
:108DC0000090019002900698069980B2049007984E
:108DD000090C02040014114307900027089D09980C
:108DE00006913E463C4603900398A9B20204000C4B
:108DF000039004982D0C154348430021224600F0AF
:108E000018F8C719714110340E46402CECDB384677
:108E1000029A00F00EF8009A019B801800905941C8
:108E200002980191103002904028CCDB00980BB0E2
:108E3000F0BD10B5202A04DB0146203A9140002005
:108E400010BD914020239C1A0346E34019439040F3
:108E500010BD10B5202A04DB0846203AD04000217E
:108E600010BD0B46D340D0402024A21A91400843A5
:108E7000194610BD10B5202A06DBCB170846203A4C
:108E80001041C1170B4306E00B461341D04020248C
:108E9000A21A91400843194610BD000000487047CF
:108EA0007445010110B50446FFF7F8FF0068005D46
:108EB000C007C00F10BD0000026813785118016090
:108EC0001846704710B5D1600449516104491162D8
:108ED00000211161114600F08FF910BDB98E00011B
:108EE000A58E00014268002A08D001680B78491C51
:108EF000002B03D0521E06C0184670470121C160E6
:108F0000881E70474268002A0BD0C3680168002B96
:108F100007D183688B4204D0491E521C06C0002032
:108F200070470020C0437047F7B582B0029C00270D
:108F30002078641C15460197302802D0002D15D0EA
:108F400015E020780127641C782804D0582802D026
:108F5000002D09D00BE0002D01D0102D07D10027E6
:108F600010252078641C02E0082500E00A25002670
:108F7000009610E00099012769430818020C294661
:108F800080B2714300908E183804864201D30120CC
:108F900001902078641C294600F01EF90028E9DAC7
:108FA0000398002805D0002F01D0641E00E0029C29
:108FB00004600198002806D002F0B8FA022101608E
:108FC000C81E05B0F0BD009930040843F9E7000061
:108FD0000FB400B589B00CA900910B990023CB60A8
:108FE000204B214A06930792042201921F4A0292C3
:108FF0001F4A089202466B460020FFF74AFA09B062
:1090000008BC04B0184770B586B006460020C043BF
:109010000190002015460C460091029104903246C2
:10902000694604A8FFF7D4FF024604982118002DD2
:1090300005D0002801D0084600E0204628600498AA
:1090400000280DD0002A02DD0098884208D0081BB5
:109050000190009432466946029404A8FFF7B8FFD5
:1090600006B070BDE58E0001058F0001FFFFFF7F98
:10907000A58E0001002904DA401C490001D14008F6
:109080004000704770B40024050C05D11024000482
:1090900002D1002921D01124050E01D1000208348B
:1090A000050F01D10001241D850F01D18000A41CF2
:1090B000002801DB4000641C002908D020252E1B5D
:1090C0000D46F540A14000D0012129430843010687
:1090D0001B1B000ADB1D02D5002070BC7047DB059E
:1090E000181880180029F8DA401C4900F5D170BC26
:1090F00040084000704710B5002B08DA0024401CDF
:10910000614192185B411A4301D14008400010BDF3
:10911000F0B51FB482B005460C0003D0084602F03B
:10912000EDF902E002F0EAF9203002460090214613
:109130002846FFF77EFE049B059A04460F46184317
:109140001143084314D0184610431BD00098402107
:109150000A1A18460599FFF77CFE05460E46009A46
:1091600005990498FFF765FE084305D0012004E047
:109170002046394607B0F0BD0020C11705430E4315
:109180002C43374300990E986305401A7905E40A89
:1091900000220C43FD0A0A3002D500200146E9E70F
:1091A0000105101969410C9C0D9D00196941FFF7DB
:1091B000A2FFDFE7064C0125064E05E0E36807CC79
:1091C0002B430C3C98471034B442F7D3FEF77CFF96
:1091D0001C4901013C4901013A2800D230382023C2
:1091E00002469A43412A01D310463738884201D3B8
:1091F0000020C04370470000F3B58DB000200A90F6
:1092000001200B90002608460C300C46099062693C
:10921000012109989047051E2ED0252D2DD0216AB9
:109220008847002818D06269012109989047216A6F
:1092300088470028F7D1411E62690998904700E0ED
:10924000761CA1690D988847216A88470028F7D1C4
:10925000E1690D988847DAE7A1690D9888470746C4
:10926000A84201D1761CD2E7E1690D9888477F1C9E
:1092700002D10A98002877D049E1002762693D466B
:109280003946099890472A280CD16269012109982A
:109290009047012506E00A214F433F18303FEBD4A9
:1092A0001020054362690121099890470146303931
:1092B0000A2903D29B498F42DEDCECE7E90600D4A1
:1092C000994F6C280AD04C2810D0682824D06A28DE
:1092D0002ED074280CD07A280AD00DE062690121C2
:1092E000099890476C2823D004211CE020200543D6
:1092F0006269012109989047A760656065284FD091
:1093000026DC582839D01ADC452849D012DC25281B
:1093100034D04128B0D143E06269012109989047D7
:10932000682802D008210D43E6E70120C002DEE7ED
:109330000220DCE7462833D047282CD130E05B28D8
:1093400070D061282CD063286CD0642823D161E0D0
:109350006F284FD009DC662822D0672820D06928E2
:1093600026D06E2817D12EE0CDE070284DD073287E
:109370006FD075284ED078280DD154E0A1690D9892
:1093800088470546252800D16CE7E1690D98884794
:109390006D1C00D16DE7BAE00A224CE00A2252E0CF
:1093A000012023466A46C0430D99FFF772F8A3E0F7
:1093B0002846402108436060A807234601D50022C3
:1093C00039E000223FE0E80700D020E72068011DD7
:1093D00021600068290501D5067018E7290701D525
:1093E000068014E7A90703D5F117066041600EE770
:1093F00006600CE72846402108436060A807234622
:1094000001D5082217E008221DE0484928460840F7
:10941000606016E02846402108436060A8072346A4
:10942000BCD5B9E715E02846402108436060A8078D
:1094300007D5234610220120C0430D99C046C046DF
:109440005AE0234610220120C0430D99C046C04671
:1094500052E000210C910B460091632802D05B285A
:1094600007D043E0E80601D40120A060012000906D
:109470003CE062690121099890475E2805D10120EE
:109480000C9001466269099890472169002906D12C
:109490000B4601AA8F00491CD3510829FADB00288A
:1094A00035D0216900290ED1C117C90E09184A11FA
:1094B000930001AA9A1849094901411A0120136829
:1094C00088400343136062690121099890475D2831
:1094D000E5D10C98002808D0002001AB81005A5833
:1094E000401CD2435A500828F8DB01AB0120224629
:1094F000C0430D99C046C04600280ADA401C06D178
:109500000B98002803D00020C0430FB0F0BD0A988C
:10951000FBE7E90702D10A99491C0A913618002095
:109520000B9074E6CCCCCC0CFFFFFF7FF1F7FFFF74
:1095300070B58D180478401CA207920F01D10278F3
:10954000401C231106D10378401C03E006780E70FE
:10955000401C491C521EF9D1002B15D002780C2654
:109560008A1A3440401C0C2C03D0A401121B9B1CF3
:1095700008E004782402121B401CF8E714780C70F1
:10958000491C521C5B1EF9D5A942D3D3002070BDE3
:1095900003B40148019001BD232A000003B401482F
:1095A000019001BD6D56000003B40148019001BD5A
:1095B0006560000003B40148019001BDAF7F000069
:1095C00003B40148019001BDB551000003B4014846
:1095D000019001BDD37E000003B40148019001BD9C
:1095E000697E000003B40148019001BDC37F000003
:1095F00003B40148019001BDE954000003B40148DF
:10960000019001BD9957000003B40148019001BDCC
:10961000ED57000003B40148019001BD1D7C00001E
:1096200003B40148019001BD0D2A000003B40148B4
:10963000019001BDAB52000003B40148019001BD8F
:10964000F58F000003B40148019001BDE1FE000068
:1096500003B40148019001BD250E010003B4014887
:10966000019001BDB143000003B40148019001BD68
:1096700085290000C943416070470268702392B297
:109680009A430A430260704770B5044601F03CFEFD
:10969000002818D08069002815D0FFF79FFA0546EA
:1096A0002046FFF79BFA2946FFF7AEF8FFF72CFBA1
:1096B000064A074BFFF704FA0022064BFFF7E6F8CD
:1096C000FFF75EFB70BD044DEAE700001F85EB511C
:1096D000B81E01400000394000803B4470B50D4683
:1096E0000646002401F010FE002816D0C1690029AA
:1096F00013D0026A002A10D08BB290B289B292B213
:10970000102D0CD0202D0AD0302D17D0402D15D083
:10971000502D13D0602D11D022E0002070BD891A89
:10972000B01AAF2292005043FEF742FD0446963431
:109730000FD47D20C000844211DC11E0191AAF2241
:10974000301A12015043FEF733FD4B21C900441873
:1097500001D5002404E0E1200001844200DD04463C
:10976000204670BD70B5104CA0421BD1851401215C
:10977000284601F07BFC0021284601F077FC0121FE
:10978000284601F067FC09486061002020606060A5
:109790001F21A16006492161A06160622062A06270
:1097A0000448E06170BD000000080240080A0200A1
:1097B0000000FC0F2E6D00000029016802D001227C
:1097C000114301E049084900016070470422002963
:1097D000816902D0114381617047914381610848DA
:1097E0000649C1620749016307494163074981632B
:1097F0000749C1630849074808607047220078009C
:1098000000080240E700E1009F00BF04190C0516A4
:1098100070206E286E2B00004008024002220029B2
:10982000016801D0114300E0914301607047C068B6
:1098300080B270470246526800200A4200D00120E0
:1098400070470000044A9068C90640094001C90EEB
:1098500001439160704700000008024010B50B48BA
:109860008CB01EC803940293019200911EC8079405
:109870000693059204914268016880680A900992F3
:109880000891684603F068FB0CB010BD0040000171
:10989000F0B58DB00E46032807DA64A004F00CF88A
:1098A0006AA004F009F86F480FE00027B4683A4650
:1098B0000BA920460B97FEF717FF05460B98A04211
:1098C00002D00078002804D067A003F0F5FF0DB0A7
:1098D000F0BD6A4C0FCC03930292019100900FCC23
:1098E0000793069205910490A268616820680A9225
:1098F00009916349009A0890203C68468A4205D144
:10990000282103F0DBFE0A9988420DD000970197C9
:109910000297039704970597069707970897099763
:1099200058A00A9703F0C8FF64A17068FEF7C7FC4F
:10993000002804D070680178622908D02BE0012D3E
:1099400003D0022D01D05FA0BFE701953BE0417835
:10995000312902D0322902D01DE002AF00E006AF6B
:1099600060A1801CFEF7ABFC002816D070685FA1D8
:10997000801CFEF7A4FC00281AD070685DA1801C32
:10998000FEF79DFC00281BD070685BA1801CFEF7D1
:1099900096FC002816D059A097E75E48854205D06E
:1099A00041208004854201D05BA08EE73D600AE043
:1099B0000720C003854201D963A086E77D6002E0ED
:1099C000BD6000E0FD602A4668A0716803F00EFFEC
:1099D0006F4E6D463078002803D101F003FB012063
:1099E0003070274800902821284603F067FE0A902F
:1099F000204601F0E5FA00280DD12C222946204608
:109A000001F00CFB002806D12C2221462846FEF747
:109A10006EFC002801D05FA057E763A003F04CFF65
:109A2000684603F099FA0DB0F0BD000075736167E8
:109A3000653A206273736574203C6669656C643EA8
:109A4000203C76616C3E0D0A000000002020666913
:109A5000656C643A20616374697665203C317C32C0
:109A60003E0D0A00D048010162737365743A2062AA
:109A700061642076616C75650D0A0000004000018C
:109A800011C011CA62737365743A20657869737482
:109A9000696E67207265636F726420696E76616CAF
:109AA00069642C2072656275696C642066726F6DE2
:109AB00020736372617463680D0A000061637469E6
:109AC0007665000062737365743A20616374697629
:109AD00065206D7573742062652031206F722032AD
:109AE0000D0A0000616464720000000073697A6509
:109AF0000000000063726300766572006273736534
:109B0000743A20756E6B6E6F776E206669656C6453
:109B10000D0A00000080000162737365743A2061D1
:109B2000646472206D757374206265203078303102
:109B3000303038303030206F72203078303130346F
:109B4000303030300D0A000062737365743A207350
:109B5000697A652065786365656473203232344BB9
:109B6000422062616E6B0D0A000000006273736533
:109B7000743A202573203D2030782530386C582CDD
:109B80002077726974696E672E2E2E0D0A00000010
:109B90008A47002062737365743A20666C6173684B
:109BA000206661696C0D0A0062737365743A206FF8
:109BB0006B20287665726966696564290D0A000064
:109BC00000B583B0002103200B46012201910090D3
:109BD000920203A1034809F0D1FB03B000BD0000CD
:109BE000434C4900ED9F000110B5022805DB486891
:109BF0000DA1FEF764FB002805D00D480078002871
:109C000004D00CA103E006F033FF10BD0BA110A09F
:109C100003F0ECFD124C13A0218903F0E7FD1CA01A
:109C2000E16803F0E3FD10BD6A736F6E0000000091
:109C30008847002076616C69640000006465666195
:109C4000756C7420286E6F742073617665642900CA
:109C5000706172616D733A2025730D0A0000000077
:109C6000A45C002020206C6564203D202575202008
:109C7000286C65643120626C696E6B2068616C666B
:109C800020706572696F642C206D73290D0A0000C5
:109C9000202070776D203D20256C7520202870775E
:109CA0006D20647574792C202525290D0A0000008B
:109CB000F3B595B015980D46032807DA6F4803F001
:109CC000FBFD6FA003F0F8FD79A023E07FA1686899
:109CD000FEF7F5FA002810D00020AE68024600908A
:109CE00069463046FEF700FD04460098B04202D0B7
:109CF000007800287BD077A00CE000240226B0007A
:109D000014902858FEF7D4FA0746E019801C502812
:109D100004D975A003F0D0FD17B0F0BD002C03D01E
:109D2000202069460855641C14983A46295868460C
:109D30000019FEF799FA1598E419761C8642DEDBC5
:109D4000002069460855451E6E462C4605F0C8FAA7
:109D5000304603F009FC060023D003F0EAFB00289C
:109D60001FD069A1304603F0ADFB074603F0D8FBD6
:109D7000002800D07D6965A1304603F0A3FB0746AB
:109D800003F0CEFB002800D07C69002D13DA002CF4
:109D900022DA5FA003F090FD304603F069FB17B0B4
:109DA000F0BD65A003F088FD002EF8D0304603F02A
:109DB0005FFB17B0F0BD294666483239814209D3AE
:109DC000654A322165A003F011FD304603F050FBD7
:109DD00017B0F0BD002C0BDB642C09DD642164A0FE
:109DE00003F004FD304603F043FB17B0F0BD14E070
:109DF000304603F03DFB002D01DB62480581002C5D
:109E000001DB6048C46006F087FE002801D05EA038
:109E100080E706F02DFE17B0F0BD3BA16868FEF7A5
:109E20004EFA002807D039A16868FEF748FA0028E2
:109E30000DD05CA06EE7204646493238884203D3F5
:109E4000454A322145A015E04E48048109E0642CC2
:109E500005D9642146A003F0C9FC17B0F0BD4948FC
:109E6000C46006F059FE002801D055A052E72246F2
:109E700059A0696803F0BAFC17B0F0BD8C48010125
:109E800020206C6564203D206C65643120626C6923
:109E90006E6B2068616C6620706572696F64203536
:109EA000302E2E3130303030206D730D0A0000001E
:109EB000202070776D203D2070776D206475747957
:109EC00020302E2E31303020250D0A006A736F6E3F
:109ED000000000006170707365743A206261642054
:109EE00076616C75650D0A00617070736574206A27
:109EF000736F6E3A206C696E6520746F6F206C6FA3
:109F00006E670D0A000000006C65640070776D00DC
:109F1000617070736574206A736F6E3A206E6F2083
:109F20006B6E6F776E206B657920286C65642C20D2
:109F300070776D290D0A0000617070736574206A76
:109F4000736F6E3A207061727365206661696C0D83
:109F50000A000000DF260000102700006C65642066
:109F600072616E67652025752E2E25750D0A00001D
:109F700070776D2072616E676520302E2E25750D0D
:109F80000A000000A45C0020617070736574206A90
:109F9000736F6E3A20666C617368206661696C0D40
:109FA0000A000000756E6B6E6F776E2070617261D3
:109FB0006D20286C65642C2070776D290D0A0000D7
:109FC0006170707365743A20666C617368206661B5
:109FD000696C0D0A000000002573203D20256C757A
:109FE0002C2073617665640D0A000000002498B08F
:109FF000F4A725461594661E38461294FEF758F9C4
:10A0000081B2384603F072F90027FF4339466846AB
:10A0100003F0CCF80028F7D01598002805D00021CF
:10A020001591694609788142EED0129801281FD017
:10A03000022826D0684600781B287DD009287CD0CD
:10A040000D287BD00A287AD0082879D07F2877D0AD
:10A05000014620395F29D7D23F2C72D2E5490855F5
:10A06000641CA4B20121684603F040F92546CBE701
:10A07000684600785B2802D000201290C4E70220D6
:10A08000FBE70020129068460078412816D042284D
:10A09000BAD1002EB8DB761E57D4D7484078801B43
:10A0A000C01DC117490F0918C908C900401A81010C
:10A0B000D24809184038FEF727F949E0CE48711C0C
:10A0C00002789142A0DA4078761C801BC01DC1172F
:10A0D000490F0918C908C900401A8101C748091861
:10A0E0004038FEF711F9C3480290FEF7E1F887B255
:10A0F000C3A42046FEF7DCF881B2204603F0F6F850
:10A100000024002D0BD9C1A00190FEF7D1F881B237
:10A11000019803F0EBF8641CA4B2AC42F3D3B8A4EA
:10A120002046FEF7C5F881B2204603F0DFF8002F85
:10A1300034D03946029805E036E038E0E2E0E3E06A
:10A1400029E136E103F0D2F828E0AA49002008709E
:10A15000A8480290FEF7ACF887B2A9A42046FEF703
:10A16000A7F881B2204603F0C1F80024002D0BD9D6
:10A17000A6A00190FEF79CF881B2019803F0B6F812
:10A18000641CA4B2AC42F3D39DA42046FEF790F821
:10A1900081B2204603F0AAF8002FCAD13D46954867
:10A1A000FEF786F884B22FE7012012902CE703F027
:10A1B0007BF8904800252F46019003F0AEFA1390EB
:10A1C000224620210198FEF788F8002860D10199E5
:10A1D00008551399149000295AD9149803F0A0FA3D
:10A1E000224616900199FEF798F8002819D1002F01
:10A1F0000AD102A81699FEF787F802A8FEF758F8C8
:10A2000085B20DE06D1EADB2A54206D92A4602A860
:10A210001699FEF782F80028F4D1002002A94855CB
:10A220007F1C14981399401C14908842D5D3002F9A
:10A2300064D0012F1AD0A5422BD902AF3F2C5DD29A
:10A24000AC425BD23819012103F050F80198395D16
:10A250000155641CA4B2F1E73819012103F046F856
:10A260000198395D0155641CA4B200E002AF3F2C97
:10A2700044D2AC42F0D3019820210155641C63A55F
:10A28000A4B22846FEF714F881B2284603F02EF84F
:10A2900034E05FA52846FEF70BF881B2284603F0AC
:10A2A00025F81398002500281CD9284603F038FA11
:10A2B000074622460199FEF730F800280ED13846AD
:10A2C000FDF7F6FF81B2384603F010F851A7384683
:10A2D000FDF7EEFF81B2384603F008F813986D1CC5
:10A2E0008542E2D34AA52846FDF7E2FF81B228461F
:10A2F00002F0FCFF2146019803F08EFA254602F099
:10A30000E3FF81E60A2000E00D20159002F0CCFF6B
:10A310003FA52846FDF7CCFF81B2284602F0E6FFB4
:10A320003449002008550D46287800281FD0324CAB
:10A33000207800280AD06078C01D4007C10D2F4842
:10A3400008182946FDF7BBFF002810D0607881016E
:10A350002A4808182946FDF7D7FF6078401C4007B7
:10A36000400F60702078082801D2401C2070002027
:10A3700003F09CFA1F4803F0DFF91CA42046FDF708
:10A3800097FF81B2204602F0B1FF02F09DFF00244A
:10A3900025463E4638E6002CB3D0641E1EA5A4B266
:10A3A0002846FDF785FF81B2284602F09FFF25462B
:10A3B0002AE61AA73846FDF77BFF81B2384602F03D
:10A3C00095FF21E60D0A434C492072656164792EA0
:10A3D0002054797065202768656C702720666F723D
:10A3E00020636F6D6D616E64732E0D0A6361696920
:10A3F000632D3E00C0500020444700200051002043
:10A400000D63616969632D3E0000000020000000BB
:10A410000D0A0000202000000820080007000000AE
:10A4200010B50C46022812DB0EA16068FDF747FF4D
:10A43000002809D00CA16068FDF741FF002804D076
:10A440000AA003F039FA10BD012001F05BFF01F012
:10A4500053FF002801D003A100E003A10AA003F0EC
:10A46000C5F910BD6F6E00006F6666007573616799
:10A47000653A20626C656C6F67205B6F6E7C6F66FF
:10A48000665D0D0A00000000626C65206C6F673A23
:10A490002025730D0A000000F8B502F0BFF9074649
:10A4A00002F0B8F90546224A22A125A003F09EF940
:10A4B0002A48874203D12AA003F0FEF915E000F0F4
:10A4C00023FF044602F0FEF906460A213846FDF74E
:10A4D0006FFE0A460146002C01D0A06900E0002072
:10A4E0000090334626A003F081F902F007FA0146F6
:10A4F0002DA003F07BF93048854203D12FA003F053
:10A50000DBF903E0294635A003F070F909F002F801
:10A510007D21C900FDF736FE014634A003F066F93F
:10A5200008F0F2FB014635A003F060F9F8BD000029
:10A530000E00010056312E30302E31340000000064
:10A540006669726D776172653A20257320283078CC
:10A550002530386C58290D0A00000000FF7F0000EC
:10A56000636869702074656D703A204144432072BD
:10A570006561642074696D656F75740D0A00000073
:10A58000636869702074656D703A2025642E2564B7
:10A59000204320286164633D2575207472696D3DF8
:10A5A000256C75290D0A00007664643A2025752013
:10A5B0006D560D0A00000000FFFF000066616E206E
:10A5C00072706D3A206E2F6120286E6F2074616367
:10A5D000686F6D65746572290D0A000066616E20F2
:10A5E00072706D3A2025750D0A000000757074694F
:10A5F0006D653A20256C7520730D0A0066726565DD
:10A6000020686561703A20257520420D0A0000001F
:10A6100002F0B4FA00280DD007A003F04DF9C820CD
:10A6200008F036FABFF34F8F11491048C860BFF3E6
:10A630004F8FFEE70FA0F0E7666163746F72793A9F
:10A6400020666C6173682077726974652066616941
:10A650006C65642C20726573657474696E67206123
:10A660006E797761792E2E2E0D0A00000400FA050E
:10A6700000ED00E0666163746F7279206465666165
:10A68000756C747320726573746F7265642C2072BC
:10A690006573657474696E672E2E2E0D0A000000B6
:10A6A00070B5194D0E46022819DB00240C206043BA
:10A6B00029587068FDF703FE002807D0641C0E2C93
:10A6C000F4D312A0716803F091F870BD0C204443DC
:10A6D00060194268295916A003F088F870BD17A0C8
:10A6E00003F0EAF8002420460C21484341194A6847
:10A6F00029580FA003F07AF8641C0E2CF3D312A093
:10A7000003F0DAF870BD000044440101756E6B6E11
:10A710006F776E20636F6D6D616E643A20257320D4
:10A7200028747279202768656C7027290D0A00004B
:10A730002020252D38732025730D0A00636F6D6D61
:10A74000616E64733A0D0A006B6579733A20544167
:10A7500042203D20636F6D706C6574652C205550F0
:10A760002F444F574E203D20686973746F72790DE6
:10A770000A00000070B50C46032823DB60680178EE
:10A78000312902D0322906D01CE04078002819D1A6
:10A79000184E012504E04078002813D1164E4025BC
:10A7A00016A1A068FDF78BFD00280FD014A1A068AA
:10A7B000FDF785FD00280ED012A1A068FDF77FFDF2
:10A7C00000280DD011A003F077F870BD294630465F
:10A7D00000F050FB08E02946304600F047FB03E05C
:10A7E0002946304600F018FB11A0A268616802F00B
:10A7F000FDFF70BD000C0140000801406F6E0000BD
:10A800006F666600746F67676C65000075736167DB
:10A81000653A206C6564203C317C323E203C6F6E92
:10A820007C6F66667C746F67676C653E0D0A00001E
:10A830006C656420257320257320646F6E650D0A96
:10A840000000000006A003F037F8C82008F020F947
:10A85000BFF34F8F07490648C860BFF34F8FFEE72D
:10A86000726573657474696E672E2E2E0D0A000072
:10A870000400FA0500ED00E010B508F04BFE7D2164
:10A880000446C900FDF77EFC0246214610A002F0F6
:10A89000ADFF08F02FF8014614A002F0A7FF08F062
:10A8A00039FA044608F030FA024605212346090326
:10A8B00011A002F09BFF1DA002F0FEFF274900201F
:10A8C0000870084608F004F9244802F0F5FF10BDAE
:10A8D000757074696D653A20256C75207469636BB9
:10A8E000732028256C752073290D0A007461736B21
:10A8F000733A2025750D0A00686561703A20746FFF
:10A9000074616C20257520422C20667265652025B7
:10A910007520422C206D696E206576657220667206
:10A92000656520257520420D0A0000006E616D6589
:10A93000202020202020202020202020207374612F
:10A94000746520207072696F2020737461636B28B6
:10A95000772920206E756D0D0A000000E04E002062
:10A9600010B506A002F0A8FFE12149020BA002F0F9
:10A970003DFF16A002F0A0FF10BD000075736172CC
:10A9800074313A2054583D5042362052583D50427E
:10A99000372028414634290D0A00000062617564A1
:10A9A0003A20256C752C203820646174612062691E
:10A9B00074732C206E6F207061726974792C203151
:10A9C0002073746F70206269740D0A00666C6F7773
:10A9D00020636F6E74726F6C3A206E6F6E653B20F1
:10A9E00074783A20444D41204348312028706F6CE0
:10A9F0006C6564293B2072783A205258444E4520B9
:10AA00006972712071756575650D0A0010B5E124D4
:10AA10006402204602F010FC214602A002F0E6FE8D
:10AA200010BD000075736172742072657365743AAD
:10AA300020256C7520384E312C2072782071756578
:10AA4000756520666C75736865640D0A000000000A
:10AA500010B506A108A002F0C9FE0DA002F02CFF5F
:10AA60001948016819A002F0C1FE10BD56312E3000
:10AA7000302E3134000000006669726D77617265B6
:10AA80002076657273696F6E3A2025730D0A000097
:10AA90006D636D2D6464632D626C653A20424C4594
:10AAA00028726474737329202B2046726565525492
:10AAB0004F53202B205541525428444D4129202BDF
:10AAC00020434C490D0A0000004000205379737464
:10AAD000656D436F7265436C6F636B203D20256C21
:10AAE0007520487A0D0A00004860704701681A4ACC
:10AAF000114001600021016041608160C160174A1E
:10AB00001749904204D148680F22104348607047AB
:10AB1000144A904204D14868F022104348607047BC
:10AB2000114A904205D148680F2212021043486032
:10AB300070470E4A904205D148680F221203104315
:10AB4000486070470A4A9042FBD148680F221204BD
:10AB50001043486070470000FEFF000008000240FC
:10AB6000000002401C00024030000240440002404D
:10AB7000580002400029016802D00122114301E07F
:10AB8000014A114001607047FEFF0000024609685B
:10AB90000020114200D001207047000030B403684B
:10ABA0000D4A0C6A13408A684D6922430C692C4394
:10ABB00022438C692243CC6922434C6A22438C6A2B
:10ABC00022431A430260CA6842600A688260496888
:10ABD000C16030BC704700000F80FFFF002B01D028
:10ABE0001061704700201061704700000149486102
:10ABF0007047000000040140054B002219685B69A2
:10AC00000140034202D0002900D0012210467047C3
:10AC10000004014010B4837919490268002B28D040
:10AC20000B6893430B604A6803689A434A60027951
:10AC3000521813680468234313608A6803689A43B0
:10AC40008A60CA6803689A43CA604279102A06D0AB
:10AC500051180A68006802430A6010BC70478A688D
:10AC600003681A438A60CA6800680243CA6010BC5D
:10AC700070470079401801689143016010BC70472B
:10AC8000000401400B680022002B56D0F0B40124D0
:10AC90000B68944023424AD04B68022B01D0122B00
:10ACA00016D113070AD5456A5307DB0E0F269E40BF
:10ACB000B5434E699E402E43466209E0056A53073C
:10ACC000DB0E0F269E40B5434E699E402E43066222
:10ACD0004B68012B05D0112B03D0022B01D0122B76
:10ACE00006D14568DB06DB0FA54393402B43436049
:10ACF0000568530003279F400E79BD43B607B60F82
:10AD00009E402E430660C5688E68BD439E402E431C
:10AD1000C66085680126A543CC6894402C438460B6
:10AD2000C46A9E400D69B4439D402543C5620B68CB
:10AD3000521CD340ABD1F0BC70477047054901604D
:10AD4000002242600F218260416101210261C160E5
:10AD500070470000FF3F00008162704781617047CB
:10AD600042694A404261704782B0EFF30884FDF7C0
:10AD7000BDF9400701D5EFF309840AA000F084FB78
:10AD8000E06800900CA0A3686268216800F07CFB7A
:10AD9000E069009014A0A3696269216900F074FB66
:10ADA000FEE700000A2A2A2A20486172644661757B
:10ADB0006C74202A2A2A0A00523020203D2530387F
:10ADC0006C5820523120203D2530386C58205232AA
:10ADD00020203D2530386C5820523320203D25302E
:10ADE000386C580A00000000523132203D253038BE
:10ADF0006C58204C5220203D2530386C5820504350
:10AE000020203D2530386C5820785053523D253055
:10AE1000386C580A0000000010B5FFF7A1FF10BD04
:10AE200030B505460E4887B00C46854202D1012157
:10AE3000042004E00B48854210D10121082000F0D5
:10AE400021F90948844209D86846FFF777FF0120B5
:10AE50000190694600942846FFF714FF07B030BD03
:10AE600000080140000C0140FF3F000010B5FFF753
:10AE700073FF10BD10B5FFF771FF10BD10B40021B6
:10AE80004156FF23CAB29207D40E4278A3409207DC
:10AE9000120EA24000290BDA0907090F08398C08A5
:10AEA0001049A4006118CC699C431443CC6107E0AD
:10AEB0008C080D49A40061180C689C4314430C6075
:10AEC000827801210078002A04D0C006C00E81409B
:10AED000064803E0C006C00E81400548016010BC72
:10AEE0007047000000ED00E000E400E000E100E059
:10AEF00080E100E0F7B5FFB004460025A5B00520CD
:10AF0000EFF31087FF210090453102A8FDF7C5F946
:10AF1000EFF31086FF21453153A8FDF7BEF953A882
:10AF2000013001909822224953A8FDF79DF9012094
:10AF300080F310880198804786F3108801221D490C
:10AF4000120303265300360388420AD194421AD0D2
:10AF50009C4201D1151116E0B44210D101256D02B9
:10AF600011E0154988420AD1944201D115460AE000
:10AF70009C4201D11D4606E03546AC4203D0009804
:10AF80007FB028B0F0BD06ACFF22013441320B493E
:10AF900002A8FDF769F9012080F310882846A69AD7
:10AFA000A599A04787F310887FB028B0F0BD0000B6
:10AFB00040390101C44013008560130000380101CD
:10AFC00010B5EFF31084012181F31088FF210906E9
:10AFD000401803490968884784F3108810BD0000B1
:10AFE0000440002010B50848064901600749416047
:10AFF00007498160C922920006490748FDF734F9E4
:10B0000010BD0000E14800200440002075490020E8
:10B0100049480020E43901014048002010B5EFF311
:10B020001084012383F31088FF231B06C018034BF1
:10B030005B68984784F3108810BD0000044000202E
:10B04000034AD16A102399430143D162704700003B
:10B0500000100240044A0029516901D0014300E078
:10B06000814351617047000000100240044A0029EA
:10B07000916A01D0014300E0814391627047000072
:10B0800000100240044A0029916901D0014300E008
:10B090008143916170470000001002400122054980
:10B0A00012060128086802D09043086070471043D8
:10B0B000FBE700000010024030B4164A5168042338
:10B0C0001940154B01D0042901D0036001E0134958
:10B0D00001605168124B8906890F5B5C0168D94099
:10B0E000416053680F4C5B055B0FE35C0D46DD4030
:10B0F000856053689B045B0FE35CD940C160D16AF3
:10B10000C90601D5084901E07D21C903016130BCB0
:10B1100070470000001002400090D0030048E80192
:10B12000D8390101DC39010100093D0070470000F8
:10B1300010B5FCF7F1FF044608F0F2F9002803D03F
:10B1400001200349000748602046FCF7E9FF10BDD5
:10B1500000ED00E010B50A4C2069411C01D0002828
:10B160000AD10120064934220003FFF7C3FE2069FB
:10B17000411C03D0002801D0024810BD002010BDA2
:10B180000C48002035480020F0B5564C85B0E069E9
:10B1900021040843E0618120534D00062863534891
:10B1A000686153482862534803220168920391431F
:10B1B0000160514934228014FFF79CFE4E4B4F4EE4
:10B1C00018694F4F411C29D0002827D0A9691A7847
:10B1D00049094901D206D20E0A43AA612168EA133D
:10B1E0009143216021687F221202914300020843AB
:10B1F00020606068304360606068B8436060606889
:10B20000211508436060206A3E4908402062206A98
:10B21000D96809020843206205B0F0BD6168204684
:10B22000314361606168B943616061680127BF02B1
:10B2300039436160002104917D21C90003910021FF
:10B2400000917F214024002502950191026861024E
:10B250008A4302600E11234908687F22120290433C
:10B26000220202430A600520FCF738FF0120FCF7A8
:10B2700035FF1C48406B800704D4284603996D1C99
:10B280008842F3D91748C06B80B2B04201D9811B04
:10B2900000E0311AB94202D2E2B28FB20292B04259
:10B2A00001D3019400E00094019A00988018C00531
:10B2B000000EA04203D0044604988142CBD809482E
:10B2C00001687F2212029143029A12020A4302602D
:10B2D000416849084900416041684907FCD405B00C
:10B2E000F0BD000000100240007000400F08000098
:10B2F00018000200001001400C480020000001006E
:10B3000000070000FF00F8FF10B50A4C2069411C3F
:10B3100001D000280AD10120064934220003FFF79A
:10B32000E9FD2069411C03D0002801D0014810BD6F
:10B33000002010BD0C48002010B501F053FF10BDD7
:10B3400010B40B06CC065B0FE40E0121A140012BCB
:10B3500007D0022B07D01430002A026805D00A4318
:10B3600004E00C30F8E71030F6E78A43026010BCC6
:10B37000704700000029818903D001225203114344
:10B3800001E0024A1140818170470000FFDF0000A8
:10B39000002A828A01D00A4300E08A4382827047F1
:10B3A0000246128800200A4200D00120704770B483
:10B3B0000A06530FCE060125F60E2A460024B24097
:10B3C000012B0FD0022B10D0838A1340090A00886A
:10B3D0008D402840002B02D0002800D001242046B8
:10B3E00070BC704783891340F0E7038AEDE70000E3
:10B3F00070B50446008A86B00D461B490840E988AE
:10B4000001432182A08919492A890840A98811434A
:10B410006A8902431143A181A08A15490840A9897C
:10B420000143A1826846FFF747FE1248844201D1DA
:10B43000039800E002982968192289005043FCF71C
:10B44000A1FE06466421FCF79DFE05012809642142
:10B450004843301A00013230FCF794FE0007000F19
:10B460002843208106B070BDFFCF0000F3E9000043
:10B47000FFFC0000003801408088C005C00D704707
:10B48000C905C90D818070470FB410B503A9044BDD
:10B49000044A029800F066F910BC08BC04B01847D2
:10B4A000ADDD0001C40100200FB410B504A9074BA5
:10B4B00002AA039800F056F9044602A9002000F001
:10B4C000F8FC204610BC08BC04B01847B3BE00010D
:10B4D0007CB51546024600201C4600290BD0491EAB
:10B4E00000920191044B6A462146284600F03AF941
:10B4F000009A002111707CBD9DBE00012021020C2C
:10B5000001D010211046020A01D010460839020964
:10B5100001D01046091F820801D01046891E42083A
:10B5200001D0881E7047081A704700000048704715
:10B530000848002030B5002805D0164C021F2068AE
:10B540000023014605E0084630BD904203D803467B
:10B5500040680028F9D1002B00D05968002B0AD090
:10B560001C68D51AA54204D11268A4181A461C609A
:10B5700002E05A6000E02260002807D01468851AB3
:10B58000A54203D1056864191460406850601846EC
:10B5900030BD000000480020F1B50E4C0F480C4EA5
:10B5A000001B0D4FC508ED0000221146009803F066
:10B5B000AFFE002803D13068002801D00020F8BD7C
:10B5C0003C6000202560606001203060ECE70000F6
:10B5D00004480020CCAD002000480020C8AF002067
:10B5E000F0B51FB486B00998089A030D00210243F4
:10B5F00014D05148514A1818504305141198012885
:10B6000010981AD0281A401C00264D4F4D4900961C
:10B6100001910490002812DA444211E011980124AB
:10B6200049A3012801D11098C1430698119A84605A
:10B630000360C26041600BB0F0BD4042E4E70446E5
:10B64000210500203F4A001C51410391029012E065
:10B65000E00707D032463B4601990098FDF7C8F94C
:10B660000191009032463B4610461946FDF7C0F95D
:10B6700006460F466410002CEAD10498039B00286C
:10B68000029A0999089806DAFDF7B2F9019B009A27
:10B69000FDF7AEF905E0FDF713FA019B009AFDF7FF
:10B6A0000FFA04460E460022284BFDF755FB03D83F
:10B6B0000020C043014607E00022254B20463146CA
:10B6C000FDF7E4F8FDF700FB102409E0002C0ADB8D
:10B6D0000A220023FCF780FD079B30321A55641EB6
:10B6E00002460A43F2D11122641C079B121B1C194B
:10B6F000119B012B03D0012308430ED10AE008431C
:10B7000004D0112010900020119077E71098151A9E
:10B710006D1E0BE01098824202DD00236D1C03E0D9
:10B72000824201DA00236D1E002BEED0069811999B
:10B730008260C16030C07EE701FCFFFF104D000059
:10B74000000014400000F03F300000000000F04313
:10B750000000E03F30380A2801D201207047002065
:10B7600070470000FFB597B00646002518E225286F
:10B7700077D100242746FD49049400E00443761C59
:10B7800032780120203A90400842F7D130782A28B8
:10B790000ED00222307801463039092916D8049992
:10B7A0000A235943303940181443761C0490F1E7BA
:10B7B000189802C804911890002904DA0120400367
:10B7C00004434842049002200443761C30782E281B
:10B7D00014D1042004437078761C2A2809D11898C3
:10B7E000761C80C8189009E00A214F43303FC719E2
:10B7F000761C3078014630390929F5D930786C2823
:10B8000010D006DC4C281AD068280ED06A2817D130
:10B8100004E0742813D07A2812D110E001204005EA
:10B8200004430CE00121090501E0032109050C4353
:10B830007178814203D1012000052418761C761C02
:10B840003078119066280BD013DC58287DD009DCA5
:10B8500000287BD04528F6D04628F4D047281AD1B6
:10B86000A5E118E0632835D0642870D0652812D18E
:10B870009DE170286CD008DC6728F1D069287BD066
:10B880006E280DD06F2806D1BAE073282ED0752807
:10B8900071D0782859D01A9A199990476D1C7EE179
:10B8A0006002400F022809D003280DD00428189800
:10B8B00001680DD00D60001D189070E11898EA170E
:10B8C00001680D604A60F6E7189801680D80F2E79C
:10B8D0000D70F0E718986A4601781172001D1890F3
:10B8E0000020507202A80090012005E0189802C8BC
:10B8F000189000200091C04361070DD5002101E0A0
:10B900000199491C0191B94212DA8142F8DB009A8F
:10B91000515C0029F4D10BE0002101E00199491CA0
:10B9200001918142FADB019A0099895C0029F5D1E5
:10B93000019904981A9B471A21463846199A00F033
:10B9400097FA0199401945180BE04FE02CE113E0FC
:10B950004EE0009800990078491C00911A9A1999B4
:10B9600090470198401E0190401CF2D12146384674
:10B970001A9B199A10E137E00A20002100900191EA
:10B980006002410F022907D0189A01CA1892C21703
:10B990009446032908D00AE01898C01DC108C900C0
:10B9A00005C91891944607E000B2C21794460429CD
:10B9B00002D140B2C1178C4600226146944506DA96
:10B9C0000A460021404291418C462D2102E021058A
:10B9D00004D52B216A461173012103E0E10701D050
:10B9E0002021F7E7029155E00A200AE0102008E044
:10B9F000102000900021042004430191082703E057
:10BA000008200021019100906002410F022907D017
:10BA1000189A01CA189200229446032908D008E017
:10BA20001898C01DC108C90005C91891944603E0C3
:10BA300080B2042900D1C0B200210291210729D58A
:10BA40001199702906D0009A1021019B4A401A438F
:10BA500005D00EE040216A461173012108E06146DD
:10BA6000014306D030216A461173119951730221A6
:10BA70000291009A0821019B4A401A430AD161466B
:10BA8000014301D1610705D530216A4611730121B7
:10BA90007F1E02911199582904D035A10E910DA94C
:10BAA0000D910DE037A1F9E76146019B009AFCF783
:10BAB00093FB0E9B8C469B5C0D9A521E0D9213704D
:10BAC00061460143F0D10D9805A9081A2030019074
:10BAD000600703D501200004844300E0012701989A
:10BAE000874201DD381A00E00020019900904118DA
:10BAF000029809180498401A0490E00306D42146DD
:10BB00001A9B199A049800F0B3F94519002706E02A
:10BB100003A81A9AC05D199990476D1C7F1C029862
:10BB20008742F5DBE0030CD521461A9B199A04984D
:10BB300000F09EF9451904E01A9A302019999047AF
:10BB40006D1C0099481E00900029F5DC08E00D9856
:10BB50000D990078491C0D911A9A199990476D1CFE
:10BB60000199481E01900029F1DC63E109280100D8
:10BB70003031323334353637383961626364656663
:10BB80000000000030313233343536373839414225
:10BB9000434445460000000000F05AF94519761C60
:10BBA0003078002800D0E2E528461BB0F0BD6007E1
:10BBB00000D406271898C01DC108C90048680A6843
:10BBC0000831C30FDB071891190001D09CA108E0D0
:10BBD000210501D59BA104E0E10701D09AA100E075
:10BBE0009AA1430011985B08109165280CD006DCDF
:10BBF000452809D046281DD0472841D141E0662874
:10BC000018D067283CD13CE00021112F01DB112026
:10BC100000E0781C0191009008A911A8FFF7E0FC52
:10BC2000139905910021119A15927F1C1298019782
:10BC3000009150E00120C00703900120019008A965
:10BC4000009711A8FFF7CCFC139A149905920022D3
:10BC5000119B009212981593059A0192002901D028
:10BC6000104602E0791C40180190381A01D501985D
:10BC700004E04042401E0090781C0190C01B0290DE
:10BC800043E0012F00DA01270021112F01DD1120EF
:10BC900000E038460191009008A911A8FFF7A0FC28
:10BCA00013990591119A002112981592009101970C
:10BCB00021070CD40599B94201DB019900E00191FB
:10BCC000012904DD159A491E515C302906D0B8427D
:10BCD00001DA011D05DA0121029115E00199491EE1
:10BCE000EDE7002805DC0099411800910199091A37
:10BCF00003E0019A411C914200DD01910099401A34
:10BD0000401C02900120C0070390200706D402992E
:10BD10000198814202DB0020C04302900020694666
:10BD2000C87707AF012103980337C907884224D099
:10BD3000022011902B201290039800280CDA404228
:10BD400003902D20129007E00A210398FCF71AFABD
:10BD500030317F1E039039701199481E11900029CF
:10BD6000F2DC03980028EFD1791E12980870307821
:10BD7000202108404530BF1E387006A8C01BC01DDA
:10BD8000039010980078002800D0012001994118F4
:10BD90000298C0170918039809180498401A401E01
:10BDA0000490E00306D421461A9B199A049800F0E7
:10BDB0005FF8451910980078002803D01A9A19994D
:10BDC00090476D1CE00324D521461A9B199A0498CC
:10BDD00000F04EF845191CE00098002807DB009998
:10BDE0000598884203DD1598405C199901E019997E
:10BDF00030201A9A904700986D1C401C00900298C1
:10BE0000401E0290002804D11A9A2E2019999047BA
:10BE10006D1C0199481E01900029DDDC05E0387891
:10BE20001A9A7F1C199990476D1C0399481E03901C
:10BE30000029F4DC21461A9B199A0498ACE600000C
:10BE40002D0000002B00000020000000000000007A
:10BE5000F8B5044600251E461746880404D405E0BC
:10BE600039462020B0476D1C641EF9D52846F8BD20
:10BE7000FFB50446002581B01E46C80301D5302712
:10BE800000E02027880404D505E038460399B04730
:10BE90006D1C641EF9D5284605B0F0BD4A68002A1D
:10BEA00006D00A68531C0B6010704868401E48603A
:10BEB00070470A68531C0B6010707047002903D04C
:10BEC000002801D0884201D1002070478268002AF2
:10BED00008D05268002A03D011604A60806841602F
:10BEE000012070478160496000200860F8E7FFB5D5
:10BEF00081B007000A9814460D4605D0002D03D0E6
:10BF0000002C01D0A74202D1002005B0F0BD0126CF
:10BF10007602002802D0E068304307E02846049902
:10BF200001F0B8FB051EF0D0E068B0430646A089DA
:10BF3000800505D4206A002802D004994968884702
:10BF4000E660214638462562FFF7B8FF05B0F0BD30
:10BF500000B599B060216846FCF79FF9042008AA53
:10BF6000D07012A0006801900B2010AAD070024679
:10BF700010A109A8FCF778F9002010AA107101217E
:10BF80005171D071917190731175D082A02010837E
:10BF90009176B42090831920C001D0830848009086
:10BFA000684603F095FC19B000BD000003160A189E
:10BFB000000000000AFFFFFF4E6174696F6E73009E
:10BFC000C5BF00017047000010B540210848FEF7CA
:10BFD00051FF08490020087000F08EF9002802D0B7
:10BFE00005A0FFF751FAF72003F0E6FD10BD0000B1
:10BFF00000080140374700205B424C455D20636FDD
:10C000006E6E65637465640D0A00000010B503F080
:10C0100083FC00F07FF940210648FEF727FF064920
:10C020000020087000F068F9002802D003A0FFF794
:10C030002BFA10BD00080140374700205B424C45F9
:10C040005D20646973636F6E6E65637465642C2034
:10C050006164766572746973696E67207265737462
:10C0600061727465640D0A0010B58CB000240094F0
:10C0700001940294039404940594069407940894FC
:10C0800009940A94FFF766F8002804D0014601A835
:10C09000FDF77EFA07E012A001886A469180418888
:10C0A000D180808810816946CC704C810A208870CC
:10C0B00012220A7303A80CA10130FCF7D5F80C205A
:10C0C0006946088418204884FF208C84F530C88491
:10C0D0000A480885684603F0BDFC0CB010BD00009E
:10C0E000010203040506000043414949432D4D4325
:10C0F0004D2D323032363039303200008813000096
:10C1000000B583B00D4900910D49002001910290C6
:10C1100069460872684603F0A1FDFFF7A5FF00F02D
:10C1200033FAFFF715FF074803F03EFB064803F01C
:10C130003BFB03F0F1FB03B000BD00004DC100016B
:10C14000C1CD0001B5C60001A9CB000101780129CC
:10C1500028D070B50025144E144C022912D00329A2
:10C160000FD103F0D9FB00F0D5F840213046FEF79F
:10C170007DFE257000F0C0F8002802D00C48FFF7C3
:10C1800083F970BD40213046FEF774FE257000F043
:10C19000B3F8002802D00748FFF776F9F72003F03C
:10C1A0000BFD70BD704700000008014037470020BC
:10C1B0003CC00001F8BF0001F8B50646244F00203E
:10C1C000388178810124481E0D463E2814D80A463D
:10C1D00031462048FCF748F81E49002048551E48C3
:10C1E00001F064FB1B4801F0A7FA0446002001F0AF
:10C1F0005DFB388900280CD1002C12D017A00090CC
:10C20000FCF756F884B2224619480099FCF72CF83E
:10C210003C81B878002819D016A0FFF735F9002422
:10C220000CE019A0EBE7315D084620385F2800D309
:10C230002E2117A0FFF728F9641CA4B2AC4201D24A
:10C240003F2CF0D3398913A0FFF71EF9F8BD000089
:10C250004C4700200055002081D80001756E6B6EA0
:10C260006F776E20636F6D6D616E640D0A00000064
:10C270007B5800205B424C455D20636C69206578EB
:10C2800065633A20220000006F6B0D0A0000000079
:10C290002563000022202D3E2025754220727370F8
:10C2A0000D0A000030B40C49098E182902D3891EEA
:10C2B0008AB200E01422094C094D63892189ED18E6
:10C2C000C91A89B2914200D911465A186281018077
:10C2D000284630BC70470000B04D00204C4700207D
:10C2E0007B5800200348002101708180C18041708B
:10C2F000704700004C4700200148807870470000DC
:10C300004C470020002800D0012001498870704768
:10C310004C47002010B505490020087088804881EE
:10C3200000F0EEFD00F05EFB10BD00004C47002069
:10C33000F3B583B00498002400287AD95B480290B2
:10C340005B4A03981178005D002904D001290BD0C5
:10C3500002291AD122E0CA286CD15649087001205E
:10C3600090800521D18017E0524B91885854491C88
:10C3700088B2908005285DD1029841780378080240
:10C38000FF211843E131884203D9002010709080CA
:10C3900084E0C01DD080022010707FE0444A454BED
:10C3A00091885854491C88B29080D188884275D1B0
:10C3B00002980022417800780D0205433E488446E9
:10C3C000E81C86B23D48002E14D93D4F6146895C79
:10C3D000090248400021030402D54000784000E0F3
:10C3E0004000491CC9B280B20829F4D3521C92B251
:10C3F000B242EBD32F4E71198A794B79110219434E
:10C40000884247D17778B07801902948761D8078A6
:10C41000002806D03346009539462AA0019A05F037
:10C4200007FB112F2AD006DC012F09D0102F31D1A4
:10C4300024E039E032E0122F20D0202F2AD124E04E
:10C4400001273F2D11D82A4631461F48FBF70CFF24
:10C450001D49002048551D4801F028FA1A4801F0EE
:10C460006BF90746002001F021FA684607700123A6
:10C470006A460320019900F02BF80BE02B46324668
:10C480003846019900F0BAFA04E02A46314601988C
:10C4900000F0F2F90648002101708180641C0498C4
:10C4A000A4B2844200D24BE705B0F0BD8355002012
:10C4B0004C4700208055002081550020FFFF0000E0
:10C4C000211000005258000040550020F9190101C8
:10C4D000FFB5D81D80B283B01D460190FB2803D95B
:10C4E0000020C04307B0F0BD214CCA202070039843
:10C4F00060700498A070280AE5702071002D04D0A7
:10C500002A46601D0599FBF7AFFEE81C83B2194F60
:10C5100019480024002B13D9184E395D09024840F0
:10C520000021020402D54000704000E04000491C98
:10C53000C9B280B20829F4D3641CA4B29C42ECD3E3
:10C540000B4949194871000A88710D488078002804
:10C5500006D000950BA0059B049A039905F068FA94
:10C560000348019900F0D4FC002007B0F0BD0000A2
:10C570008057002081570020FFFF0000211000009D
:10C580004C4700205458000000B587B000200190AF
:10C590000090039004906A46069010730C49029133
:10C5A00005219170032313701023D3705070107104
:10C5B0000123537190715073064805907D2091734B
:10C5C00000011082104604F00FF807B000BD000013
:10C5D00040E2010000B0030110B5024803F0ACFDD9
:10C5E000002010BD544E00202F48007900285AD159
:10C5F000F8B56D202C230322072140010BF49CD2B7
:10C60000A0210446017029480027C1786170277174
:10C610000321E1806772012666710721244D21778D
:10C62000A9796177687B002803D0E78003206071D7
:10C630000EE0E87900280BD0A879022800D16677AF
:10C640002671E6802046A9792030417086700770F7
:10C6500015488079022804D0032815D004281BD15E
:10C6600016E003F0B3FF00280BD00520E0806771CF
:10C67000688A6061688AA06120460A3003F0D4FDB0
:10C680000AE0094903208871288B6061288B02E049
:10C69000E88B6061E88BA061034806714671204613
:10C6A0000BF486D2F8BD7047B04D0020344E002008
:10C6B000A04E002010B584B00A23032207211048A1
:10C6C0000BF43AD21B2101700021417014244480E4
:10C6D00003228280C1800B4A02810BF469D2684632
:10C6E000048009480190684603F080FA6846048196
:10C6F0000648039002A804F0F1FD04B010BD00004C
:10C700001B0D0000FF0100001843010179DA000150
:10C71000FFB585B0054602A800901C46284606993C
:10C7200003F0ACFF6846007A002866D006980090B7
:10C73000280A334A019403900E2826D03148002459
:10C740000178002951D92F48E100081882880399FF
:10C750008A4240D1009A81689646019A28469446BA
:10C760000A791206120E36D00968254BD700083F09
:10C77000CE1937887668BFB2874201D09F4226D152
:10C78000634603227146B04725E01F49681809280F
:10C790002BD800981D49844608792E46000623466A
:10C7A000000E1ED0C4000F68083C3C19278864683E
:10C7B000BFB2B74201D0974204D103226146284656
:10C7C000A0470EE0401E0006000EEBD109E0521E0D
:10C7D0001206120ECAD10B48641C0078E4B2A042C3
:10C7E000B1D86846007A002807D00948426C002A70
:10C7F00002D0284606999047002009B0F0BD0000FD
:10C80000FFFF00005C4D0020EEF1FFFF683E0101DC
:10C81000B04D002000487047FFFF000070B5124D7A
:10C8200001212846FCF7FAFF142006F031F97020A8
:10C8300002F07CFC702002F079FC044600212846BE
:10C84000FCF7ECFF094844800948844201D14010BC
:10C8500070BD2046FCF718FF0649FBF7D9FFFCF72F
:10C86000F5F900B270BD00000008024084470020C6
:10C87000FFFF000000002041F0B5074600208BB00C
:10C8800015460E46002A04D0012D04D13178FF2927
:10C8900001D10B4E06250024002D08D90146325D3A
:10C8A000684602F079FC641CA4B2AC42F6D303469D
:10C8B0006A4639462120FFF70BFE0BB0F0BD0000A1
:10C8C000EC44010101484088704700008447002083
:10C8D00070B506460020074D044601462A5D06480D
:10C8E00002F05AFC641CA4B2062CF6D33080024835
:10C8F00070BD0000EC4401017B5C002010B560209D
:10C9000002F014FC0449884201D1002010BD6021CE
:10C91000FCF7E4FE80B210BDFFFF000010B503F08D
:10C92000D1FB04480169002901D004208847002078
:10C9300010BD0000C04E002070B5224C606B224D2F
:10C94000C00722D0A06B21497E2209685143401ABA
:10C950002988491E29804B21C90040181C4988425A
:10C9600013D300202880206A400840002062194923
:10C9700008680204930F184A01D0904300E0104366
:10C9800008601648407F03F0D5F829880120002967
:10C99000216B07D0014321630522032110480BF4CA
:10C9A0008DD30DE0FF22120291432163216B0522FA
:10C9B000920211432163216B0143216303F054FE72
:10C9C000002070BD00100240344700208C00002081
:10C9D000B10400000010014000C00000104E002013
:10C9E000010F000004480021017041618161C161B3
:10C9F000016281627047000058470020F8B5144674
:10CA00000D46102809D0112878D0122804D11A46D2
:10CA10002146284603F042FFF8BD00910C2B04D0BC
:10CA2000002301221021284664E02278E178104694
:10CA30006278090612021043A278120410430843D8
:10CA40000502E0782D0A0006227905431046627936
:10CA5000E17912021043A279090612041043084337
:10CA60000602E079360A00060643082021180A78F3
:10CA700010464A78120210438A78C978120410438B
:10CA8000090608430702E07A3F0A000607431E48EA
:10CA90001E494124A404884202D0A0420BD10C4676
:10CAA0001B49281F88420DD3002303221021009820
:10CAB00003F0CAFFF8BD002302221021009803F002
:10CAC000C3FFF8BD13484078002804D1FEF78AFA66
:10CAD0001049012048700F48012101700021416177
:10CAE0008161C16101628162001DF0C00B460A468E
:10CAF0001021009803F0A8FFF8BDFFE71A46214671
:10CB0000284603F01FFEF8BD0080000100800001F0
:10CB1000FD7F03005847002000487047A45C0020B8
:10CB2000F8B5342211491248FBF79EFB104C114F07
:10CB300020680125104EB8420BD16068012808D149
:10CB40002046302100F0BAFD216B884201D13570BA
:10CB5000F8BD34210648FBF7A0FBFF202760F53025
:10CB6000656020810020E0603070F8BD0060000149
:10CB7000A45C00207ADA12CA8847002010B534215C
:10CB80000748FBF78AFB064806490160012141601E
:10CB9000FF21F53101810021C16003F0BDFF10BD0F
:10CBA000A45C00207ADA12CA10B584B014230322E0
:10CBB000072112480AF4C0D71B21017000214170DF
:10CBC0004724448003228280C1800D4AC2600D4AFE
:10CBD00002610B2202720AF4EBD7684604800A480D
:10CBE0000190684603F002F8684604810748039004
:10CBF00002A804F073FB04B010BD00001B0D000080
:10CC0000384301012843010120430101E5210101CD
:10CC100000207047F8B5184D184FE879002801D06A
:10CC20002E7B00E0FE780322331D072114480AF40E
:10CC300083D7A921044601701248C1786170002190
:10CC40006180E8791049002803D02A7B896C201D77
:10CC500002E0FA78201D091DFBF706FB608802211F
:10CC60008019608007480279062A00D0017141715D
:10CC700020460AF49DD7F8BDA04E0020804E00202B
:10CC8000A60D0000B04D0020604E0020F8B51F2614
:10CC900023230322072128480AF44ED70446AA205A
:10CCA000264F2070F878264D6070E8786080EA782A
:10CCB0002449201DFBF7D8FA6288B01AC1B2201DA2
:10CCC0001018214A0326032910D92B79002B0DD0E7
:10CCD0000670192343705389091F1B0AC370937A86
:10CCE00083706388C9B21B1D6380001D02291AD995
:10CCF0006B79002B17D0137B891E8B4200D219460B
:10CD0000CDB2691C0170117BA94201D1092100E05B
:10CD1000082141702A460D49801CFBF7A5FA60885E
:10CD2000AD1C401960803879062800D03E717E71B4
:10CD300020460AF43DD7F8BDA60D0000B04D0020F6
:10CD4000A04E0020844E0020344E0020414E002092
:10CD500070B53A230322072116480AF4EDD6A42120
:10CD6000154D04460170E8786070A97913480022D7
:10CD7000022910D0032913D0042916D06280227111
:10CD8000807902F007FB0520287104206871204695
:10CD90000AF40ED770BD018A642359436180EEE71F
:10CDA000C18A642359436180E9E7818B6423594335
:10CDB0006180E4E7A10D0000B04D0020A04E0020EE
:10CDC00070470000FFB50F4683B00021009101912C
:10CDD00016466946FCF7E2FB040030D10521C90282
:10CDE0006846FCF7E1FB002828D121496846FCF79A
:10CDF000DBFB002822D11F496846FCF7D5FB002841
:10CE00001CD11D496846FCF7CFFB002816D129210B
:10CE100009026846FCF7C8FB00280FD1174968468D
:10CE2000FCF7C2FB002809D115496846FCF7BCFB9A
:10CE3000002803D100988088C10B03D00624204627
:10CE400007B0F0BD00050099000D0D186888B042CC
:10CE500000D207242988B819884201D90D24EEE7A9
:10CE6000A8193A46001D0699FBF7FEF96F80E6E720
:10CE70000128000003280000022800000229000009
:10CE8000032900001EF48CD200F00EF8012005F0FA
:10CE9000FFFDF7E710B503490020087000F004F823
:10CEA00010BD0000464700201248002100780028ED
:10CEB0001FD070B5104D86B02878002817D1A888EB
:10CEC0006C88A04213D00D4E6A4680B2A04209D0B1
:10CED000335C5354401CC005491CC00D89B2A88066
:10CEE0001429F2D301202870104605F07FF906B00E
:10CEF00070BD704737470020464700200053002090
:10CF0000024900204880888008707047464700200A
:10CF1000F0B484460D480078002814D0002200297F
:10CF200011D90B480B4D878843881C465B1CDB05D9
:10CF3000DB0DBB4207D06646B65C521C2E5592B242
:10CF400043808A42F0D3F0BC70470000374700208E
:10CF5000464700200053002010B5044600681949D8
:10CF6000884208D12046282100F0A8FBA16A884207
:10CF700001D115A200E016A21B491CA000F036FC4E
:10CF800021A0216800F032FC26A0616800F02EFC90
:10CF90002AA02369E268A16800F028FC33A0616937
:10CFA00000F024FC37A0236AE269A16900F01EFCAE
:10CFB0002EA0616A00F01AFC3EA0A16A00F016FCE7
:10CFC00010BD000011C011CA76616C6964000000D8
:10CFD000494E56414C49442028626164206D616786
:10CFE00069632F637263290000400001626F6F74F0
:10CFF00073657474696E6720402030782530386C12
:10D00000583A2025730D0A0020206D61676963205E
:10D010002020202020203D2030782530386C580DED
:10D020000A00000020206163746976655F62616EAA
:10D030006B203D20256C750D0A00000020206261E8
:10D040006E6B313A20616464723D30782530386C03
:10D05000582073697A653D256C75206372633D3095
:10D06000782530386C580D0A000000002020202060
:10D0700020202020207665723D30782530386C588D
:10D080000D0A0000202062616E6B323A20616464F8
:10D09000723D30782530386C582073697A653D25AB
:10D0A0006C75206372633D30782530386C580D0AFA
:10D0B00000000000202063726333322020202020F3
:10D0C00020203D2030782530386C580D0A000000B3
:10D0D00030B58DB001210820FDF7D4FF0121880370
:10D0E000FDF7D0FF02A8FDF729FE402002900220A4
:10D0F000284D0424039002A907942846FDF7C2FD99
:10D1000080210794029102A92846FDF7BBFDE1208A
:10D1100040020890002069468884C8840885888574
:10D120000C2048851C4D08A92846FEF761F901210D
:10D130000846FDF78FFF194C2046FDF7D7FC012369
:10D14000224617490220FDF749FD01228021284689
:10D15000FEF71EF900220121402005F01BFE114CB4
:10D160002060012005F004FE606001220E4928467F
:10D17000FEF7E6F81C20694608700320487001207D
:10D1800088706846FDF77AFE01212846FEF7F2F81E
:10D190000DB030BD000C01400038014008000240D5
:10D1A00000000240384700202505000070B5054604
:10D1B0000B480468002C0ED0481C0ED008467D2178
:10D1C000C9004843FAF7DEFF02462946204605F02B
:10D1D00048FF012800D0002070BD0020C043F3E7C5
:10D1E0003847002010B582B00020104C00900E4946
:10D1F0002046FEF7DCF8002814D02046FEF73CF964
:10D20000694608710A480068002804D00A460023CD
:10D2100001A905F0DFFE0098002803D00120054990
:10D220000007486002B010BD25050000003801402D
:10D230003847002000ED00E030B5184D85B00446B9
:10D2400040212846FEF7ACF80028F9D000212846F6
:10D25000FEF790F80020694600948880C880088115
:10D2600088810C2048812846FEF7C2F80C4C2068C3
:10D27000002807D006F03EF9022803D100212068DB
:10D2800005F0AAFD012207492846FEF759F80121B9
:10D290002846FEF76FF805B030BD000000380140A9
:10D2A000384700202505000010B5064C60680028AE
:10D2B00007D006F01FF9022803D1C11E606805F0EF
:10D2C00071FF10BD3847002010B5074C606800287A
:10D2D00009D006F00FF9022805D100231A46194695
:10D2E000606805F0B0FD10BD3847002000283FD031
:10D2F00000293DD0F0B51F4E0C4605468BB00021ED
:10D300003046FDF737FC1C4F02203946FDF7ECFB99
:10D310001A4800901020029000208021059104906E
:10D320000321019503940903069007900890099141
:10D330000A9069463046FDF731FC01213046FDF781
:10D3400019FC39460220FDF721FC0028F9D0002104
:10D350003046FDF70FFC39460220FDF7C5FB084CAF
:10D3600040212046FEF71CF80028F9D00BB0F0BD94
:10D3700070470000080002400000024004380140ED
:10D380000038014010B4002807D00368002B04D0F7
:10D3900042688168914201D206E0002010BC7047CB
:10D3A000491C8160002804D0914202D25C5C202C90
:10D3B000F6D99142F2D1491E816010BC704700003D
:10D3C000F8B50C4605461046194600F013F8064617
:10D3D00000200090064B324621462846FEF787FD86
:10D3E0000028304602D100F043F80020F8BD0000CC
:10D3F0009447002070B505460E46124800F0A2F88A
:10D4000004001CD0E6610820A561E0600E4A0F4BC5
:10D4100028463146FBF7A0FC02D80D4860610EE0BB
:10D4200000220C4B28463146FBF782FC02D8012033
:10D43000C00703E028463146FBF722FC6061204626
:10D4400070BD0000944700200000C0FFFFFFDF41D7
:10D45000FFFFFF7F0000E0C110B5044800F072F844
:10D46000002801D04021C16010BD00009447002079
:10D47000002824D0F8B5124E04460027A08925685C
:10D48000C0050DD4A068002804D0FFF7F1FFA089E3
:10D49000C00505D42069002802D07168884727613B
:10D4A000A089800505D4206A002802D071688847C9
:10D4B00027627168204688472C00DFD1F8BD70478D
:10D4C0009447002010B5002201F088FD10BD000037
:10D4D00030B4124A0E4D0F4B0F4C0028136013D07E
:10D4E0000168002900D0116054604068002800D015
:10D4F0005060002090601068984203D15068A042AC
:10D5000000D1956030BC70479560546030BC704766
:10D510002926010199B5000135B500019447002085
:10D52000002803D0007B082801D00020704701208C
:10D530007047002803D0007B402801D000207047AE
:10D540000120704710B501682820884700280AD0BC
:10D550000021016041608160C160016141618161C0
:10D56000C1610162416210BD70B5002604463546B6
:10D57000002808D0FAF79CFE411C2B463246204674
:10D5800000F004F870BD002070BD0000FFB500245D
:10D5900089B006460094019434480294039404949C
:10D5A00005940694046015464460002E5AD0002964
:10D5B0003FD0024600960191D168906812690490AC
:10D5C000069205912A48FFF7BDFF0790002830D04A
:10D5D00000986F46002802D00298002801D0002051
:10D5E0000DE00198042809D9032222A10098FAF736
:10D5F00094FE002802D10298C01C02903846FFF722
:10D60000C1FE0146079803F0EDFB00280ED00C98F0
:10D61000002814D06846FFF7B5FE029901988142B0
:10D6200004D202990098405C002808D00798FFF7C0
:10D630001FFF0199029888420AD204460BE0002D90
:10D6400003D0029900984018286007980DB0F0BDEB
:10D65000081E00D0441E002D01D030192860034858
:10D660000660446000200DB0F0BD00008C47002033
:10D6700094470020EFBBBF0010B5024A002103F021
:10D68000CFFE10BD944700200149496808470000BB
:10D6900094470020002810D070B50E460446FAF7D3
:10D6A00007FE401C336805469847061E04D02A46EC
:10D6B0002146FAF7D9FD304670BD7047002230B4DC
:10D6C000D243491E0FD3094C03785A400023401C13
:10D6D0005508D20700D022465B1C6A40DBB2082BFB
:10D6E000F6D3491EF0D230BCD04370472083B8ED4A
:10D6F00002468B880020022B01D00D207047C9887C
:10D70000002A05D00029F9D00129F7D081207047DF
:10D710000029FCD00229F9D170470E207047000083
:10D720000E2804D20C2148430249085870470020B3
:10D73000704700004444010170B588B000246A4677
:10D74000234616E0401C01782029FBD00929F9D096
:10D750000906090E12D0A1005050641C00E0401CC4
:10D76000017800290AD0202901D00929F7D10370B6
:10D77000401C0178002901D0082CE4DB002C14D0D7
:10D78000104E002528460C21484331580098FAF7DE
:10D7900096FD00280CD06D1C0E2DF3D30AA0009925
:10D7A00000F024F8012008B070BD002008B070BD62
:10D7B0000C204543A81982686946204690470020FE
:10D7C00008B070BD44440101756E6B6E6F776E20BA
:10D7D000636F6D6D616E643A2025732028747279D1
:10D7E000202768656C7027290D0A00000FB410B55A
:10D7F00003AB60210648029AFDF76AFE0549002046
:10D80000C877034800F058F810BC08BC04B01847AB
:10D8100060500020A0500020F3B581B00D46019863
:10D82000FAF746FD144C86B22046FAF741FD81B264
:10D830002046FFF75BFD0024002D0BD90F4F384623
:10D84000FAF736FD81B23846FFF750FD641CA4B2EA
:10D85000AC42F3D3084C2046FAF72AFD81B22046A9
:10D86000FFF744FD002E03D031460198FFF73EFD3F
:10D87000304603B0F0BD000000A400010CA400017C
:10D8800030B40125074B084CAD0203E06254491C3B
:10D890001981401C0278002A02D01989A942F5D3C7
:10D8A00030BC70474C4700207B580020014908607D
:10D8B000704700004047002010B50749096800295B
:10D8C00001D0884710BD0446FAF7F2FC81B2204629
:10D8D000FFF70CFD10BD000040470020F0B51FB45D
:10D8E00005460398144646000198760847007F08CD
:10D8F000334628463946FBF72FFA02D228463946E6
:10D9000001E0204631463322D243FBF751F9064667
:10D910000F4622462846039B0199FBF75BF8490016
:10D9200049083B463246FBF703FA02D8012005B00E
:10D93000F0BD002005B0F0BD02460020802901D9CD
:10D940008D207047062A06D0072A07D0082AF8D16A
:10D950000729F5D170470829F2D170470629EFD37E
:10D9600070477047704770B5C46805466068002806
:10D9700003D00020002802D00CE00120FAE7201D8F
:10D98000FBF718FE09F4C8D76068002808D000200B
:10D990000028F4D00020E860204609F4BDD770BD0F
:10D9A0000120F5E730B40446A2890920521C93B245
:10D9B000E48900222546D540ED0707D05D1C8D4245
:10D9C00002D130BC104670479B1C9BB2521CD2B295
:10D9D000092AEFD330BC7047FFB585B00E9D0446D1
:10D9E0002F8801201E4600213A46CA40D20704D0A3
:10D9F0004B0003225B1C9A401043491CC9B2092901
:10DA0000F2D3049030461E210840218A184A002390
:10DA10000191009302920390132304AA15490698DA
:10DA2000FBF7CEFD009000281FD10121142009F43E
:10DA3000FDD70746E06006980188B9812988F981F9
:10DA4000F00701D00120C003079908433880208ADD
:10DA5000788014206082204600F060F8381DFBF7C3
:10DA6000B5FD208A00210AF437D1009809B0F0BD35
:10DA7000283D01010A18000000487047C03D01011F
:10DA8000FFB5087881B00C46092836D2142003F07F
:10DA9000F1FB0746217800F0EFF800282BD06178E1
:10DAA0002078FFF749FF060028D17D68002D0ED0B1
:10DAB00020782979814207D12946381DFBF78CFD52
:10DAC000284609F429D702E02D68002DF1D16078AD
:10DAD0000121083009F4AAD705462078287160781A
:10DAE00068716278A11CA81DFAF7BEFB2946381D93
:10DAF000FBF778FD02E0822600E08126022306483B
:10DB0000039A04990AF418D02178017046700AF437
:10DB10004FD0002005B0F0BD0114000010B5044640
:10DB2000142003F0A7FB0449216003216181123016
:10DB300060600120208110BDD03D0101F8B517467D
:10DB40000C4610460AF4B6D0012831D1142003F057
:10DB500091FB0546017C00F08FF80646297C22786F
:10DB60001448914214D1697C637809023A46891DB0
:10DB70009B1D09F4E1D705460680002028716078D6
:10DB800068806278A11C681DFAF76EFB284609E0E0
:10DB9000697C062309023A46891D09F4CDD706801F
:10DBA000802101710AF404D0002138460AF494D08F
:10DBB0000020F8BD140C0000F8B50F4600240978C9
:10DBC0001846254609291DD20B007B441B79DB181A
:10DBD0009F440407101313130A160D00052414A5FF
:10DBE00010E00A2414A50DE0082416A50AE0072475
:10DBF00017A507E00A2418A504E0052419A501E0EB
:10DC000006241AA50146A31C1A4809F495D706460E
:10DC1000387830707470002C04D022462946B01C2D
:10DC2000FAF722FB304609F4C3D70020F8BD000004
:10DC30004E53494E470000004E532D424C452D3166
:10DC40002E300000123456FFFE9ABCDE00000000A9
:10DC5000025E044000000300312E302E302E302DA5
:10DC60004C450000312E302E30000000FFEEDDCCA0
:10DC7000BBAA00000314000010B48289C489521C9E
:10DC800093B200222046D040C00706D0914202D174
:10DC90005B1C9BB205E09B1C9BB2521C52B2092A32
:10DCA000F0DB092A02D010BC1846704710BC0020D7
:10DCB0007047000070B5050005D0134E30688542EE
:10DCC00003D1002070BD72B6FEE704F099FE6C69C6
:10DCD00004F0A2FE7068844202D0B068844201D190
:10DCE000022070BD0948844204D1A86A0028F7D1F7
:10DCF000032070BD0648844203D0002C01D00120CF
:10DD000070BD042070BD0000A4470020B45D002059
:10DD1000A05D0020002802D00368002B01D1002064
:10DD20007047F8B50D4641680446002902D0A06846
:10DD3000884211D21B4EB5420ED8A2686D1C5019F4
:10DD4000814201D39818F8BD2169002904D11649F0
:10DD5000884203D9B04202D90020F8BD4600226AA9
:10DD60000027002A05D0314618469047050012D0FA
:10DD70000CE0A1693046884705000CD0A2682168F4
:10DD8000521CFAF771FAE1692068884766602560DD
:10DD9000A0684019F8BDE1692068884767600020E5
:10DDA0002760F8BDFFFFFF7FFFFFFF3F70B50D4D00
:10DDB00004460A2809D10D212846FDF761FB802180
:10DDC0002846FDF7EDFA0028F9D0E1B22846FDF724
:10DDD00057FB80212846FDF7E3FA0028F9D02046BA
:10DDE00070BD000000380140F0B50878324F334D67
:10DDF000334E801E83B00C46062859D20100794468
:10DE0000097949188F4402255434543A012030705E
:10DE1000A0786876A078C00705D02A492A48FBF781
:10DE2000B7FB387AA874B28A002A06D0FF20F530F2
:10DE30007080032125480AF441D1F169002937D0C7
:10DE400000200090019005206A46107068468847BF
:10DE50002EE000246C7601F0E7FDF169002927D05F
:10DE6000009406206A4601941070684688471FE0B7
:10DE70001722A11C1648FAF7F7F919E0B878000143
:10DE8000C0194030807D002812D11C22A11C1148ED
:10DE9000FAF7EAF90F48A18A0182E18A4182218BCF
:10DEA0008182618BC1820B49608A0883207F6874FC
:10DEB000002003B0F0BD0000B04D0020F44C002065
:10DEC000104D0020B94D0020074D0020040F000028
:10DED000EE4C0020D44C0020F0B518460D4601460B
:10DEE00085B022230322744809F426D60121044672
:10DEF000417028780B286ED20100794409794918BD
:10DF00008F4405CDCDCD6F6ABB23CDCD6C000120F4
:10DF1000207060706948817921710179A170C1799F
:10DF200061714179E170017AA171417AE171817A7F
:10DF30002172C16900294ED00020009002206A465B
:10DF40001070684601948847A9E0072020700120DE
:10DF5000607068461DF482D3019F009EFAF772F943
:10DF6000801960820025FAF76DF981196019009017
:10DF70008170FAF767F9C11900986D1CEDB201754F
:10DF8000082DF0D30825FAF75DF9B9194018611981
:10DF90006D1CEDB28870102DF5D310202077484805
:10DFA0008178090108184030807D012877D11C2232
:10DFB000A11C4448FAF758F94248A18A0182E18A33
:10DFC0004182218B8182618BC1823E49608A0883B4
:10DFD0003D48217F417462E0052000E00A20207066
:10DFE0005DE0042222706878012804D0002802D065
:10DFF000022833D053E00120304D6070287C002887
:10E0000010D002A81DF42AD3FAF71CF92F49FAF709
:10E01000B9F82F480818029940182E49FAF7B2F8B3
:10E02000009101E0E8680090E969002907D000202C
:10E03000029003206A46107202A8039288471021BA
:10E04000A01CFAF72AF90098A0700098000AE07066
:10E050000098010C2171000E607120E01748C16921
:10E06000002905D000200090019068460270884782
:10E0700020460C3809F492D514E00620164D207085
:10E08000E878012811D01021A01CFAF706F9A98818
:10E090006182E988A1822989E182002020762046D8
:10E0A00009F486D5002005B0F0BD10220B49A01C54
:10E0B000FAF7DAF8EBE70000140E0000104D00202C
:10E0C000B04D0020D44C0020F44C0020A0BB0D002B
:10E0D000A08601003F420F00344E0020BF4D0020BB
:10E0E00000B5084883B0026C002A08D000200090D8
:10E0F000029005206B4618706846019190470020F9
:10E1000003B000BDB04D002010B584B0FF2B19D076
:10E11000144C226C002A08D00020009002900620A7
:10E120006B461870684601919047032009F4C2D5E8
:10E13000032814D1A26F002A11D003210A4809F440
:10E14000BDD70CE009480123007F032201020848E3
:10E15000083109F4F1D40721017009F429D5002010
:10E1600004B010BDB04D0020090E0000104E00207C
:10E17000050E0000FFB5180A4C4E83B00C46B07077
:10E18000FF287DD00102342303224948083109F4D5
:10E19000D3D40546B078002701018919403188722F
:10E1A000B07821880001801940300181B078617A0F
:10E1B000000180194030C172B07862890001811974
:10E1C00040318A81A289CA81E0890882207C0128A5
:10E1D00002D0002807D00BE0B1780120090189198D
:10E1E0004031887504E0B0780001801940308775AF
:10E1F00020883080607A307221460A312D48FBF742
:10E20000C7F902F0E3F900281BD0607A012804D195
:10E2100003221146284809F4DFD402F0DFF905286B
:10E220000FD201007944097949188F440606060285
:10E23000060001202821485505E0052128204155E8
:10E2400001E0282047550321059809F445D51720FA
:10E250003086B17809018919403148821748C06871
:10E26000002803D00321164809F488D61548028DEA
:10E27000002A03D00321144809F420D7306C00E0B1
:10E280000EE0002808D00220694600970870029529
:10E290000194316C68468847284609F489D401E026
:10E2A00001F03AFB002007B0F0BD0000B04D0020A7
:10E2B000020E0000B94D0020150D0000C04E0020D8
:10E2C000030F0000344E0020020F000030B5180A82
:10E2D000144D00010C46401983B0FF21403081727B
:10E2E00001F0EEFB002803D10221032009F4F4D44D
:10E2F0002A6C002A08D00020009002900320694672
:10E30000087068460194904710210748F9F7C5FF47
:10E3100006480068002802D0092009F4C7D200206E
:10E3200003B030BDB04D0020CF4D0020100C0020B8
:10E3300000B5084883B0C169002907D000200090CB
:10E34000019009206A46107068468847002003B093
:10E3500000BD0000104D0020FFB591B00D46122306
:10E3600003224348149909F4E7D3002104460170BD
:10E3700040480078002862D03E48407C002833D0D6
:10E380003C216846F9F789FF01F012FF002841D0CF
:10E3900004A90F913749461EF0B23A2289695043C9
:10E3A00041186846091DF9F75FFF6846008B298808
:10E3B000884206D10822A91C0F98F9F798FF002877
:10E3C0000BD0207800280BD008A8407C6074102265
:10E3D0006946601CF9F748FF1CE001202070F3E754
:10E3E0003006000ED6D12AE023482988008B8842C7
:10E3F00025D10822A91C2148F9F779FF002809D165
:10E40000012020701E481022407C60741A49601C54
:10E41000F9F72AFF2078002811D01648C169002991
:10E4200007D000200090019007206A4610706846CF
:10E430008847204609F4BCD3002015B0F0BD0D4834
:10E44000C169002907D000200090019008206A4689
:10E45000107068468847022303220A48149909F479
:10E460006BD3012101700621417009F4A1D3E0E7CB
:10E47000180E0000104D0020D44C0020E44C002069
:10E48000F44C0020040E000070B50C4609781B48BF
:10E490001B4D1E46002904D0012912D002292BD180
:10E4A0001AE01C23314609F447D306462078307021
:10E4B000287B70802A7B1349301DF9F7D5FE304642
:10E4C00007E00A23314609F437D3217801706989BE
:10E4D000418009F46DD30FE00A23314609F42CD3AF
:10E4E00021780170298C4180698C8180A98CC18040
:10E4F000E98C018109F45CD3002070BD0B0E000093
:10E50000344E0020414E002010B5087800F042FF44
:10E51000002010BD05480A8842861A0A1201101808
:10E52000098840308182002070470000B04D0020F3
:10E5300030B5180AC043000683B00D46000E21D046
:10E54000190A0902E120062303220001083109F417
:10E55000F3D204460120207002206080FF20413069
:10E56000A0800B48026C002A08D0002000900420F4
:10E57000694608706846019502949047204609F460
:10E5800017D301E001F0C8F9002003B030BD00004E
:10E59000B04D002000B5084883B0026C002A08D0B6
:10E5A00000200090029008206B4618706846019188
:10E5B0009047002003B000BDB04D002070B5184654
:10E5C0000C46014602230A4809F4B6D20546094919
:10E5D000A07808736288211D0748F9F745FE0020DE
:10E5E000687020782870284609F4E2D2002070BDB7
:10E5F0000D0E0000344E0020414E00204A780B489A
:10E60000002A05D02030012A08D0022A09D00AE0C9
:10E610000279012A07D10978C17004E009780175EF
:10E6200001E009784175002070470000B04D0020DE
:10E6300070B54878002806D0FF25124C01280BD071
:10E64000022816D01BE010480179062917D10721AE
:10E65000017101F0CFF812E0207DFF280FD001F00A
:10E66000C7F90A4825750169002908D000208847A4
:10E6700005E0607DFF2802D001F09CF9657500205F
:10E6800070BD0000D04D0020B04D0020C04E0020D5
:10E6900010B5032B06D010220548891DF9F7E4FDBB
:10E6A000002010BD0348017A034801F037FEF7E768
:10E6B000CF4D0020B04D0020B94D0020F0B50D46E3
:10E6C0000878E34EE14934464978002720348DB07C
:10E6D000A1287AD012DCDF490C911B2876D006DC09
:10E6E000012819D003287CD017286DD14FE12828A4
:10E6F0006ED091286DD0A02866D152E10246A23A90
:10E70000092A61D213007B441B79DB189F44FE5C0D
:10E71000FDFD5CFDFCFDFD006878002854D1012062
:10E7200002F00CFE01F038FE342303220721CA4810
:10E7300009F402D203210170C84904468A78427064
:10E740000122C276FB224284C54AC284C54A828421
:10E750000A88028487768A888280CA88C2800A8969
:10E760002281487A8009032805D188780522104241
:10E7700001D10120A076A07E04221043A076BA48E1
:10E780006080C878012825D0204610210A30F9F78A
:10E7900084FD316C002907D001206A460097107073
:10E7A0006846019502948847012000F0F3FD204659
:10E7B00009F4FED1012303220721AC4809F4BCD19E
:10E7C0001A21017009F4F4D133E11EE1CAE008E036
:10E7D00069E049E0204610220A300C99F9F744FD1F
:10E7E000D7E7009701970297039704970597069735
:10E7F0000797089709970A970B9701F0E7FE0028FB
:10E8000005D0684601F028FD0AA801F0F5FC01F0EA
:10E81000DDFE00280CD068468079002808D108A8C1
:10E82000807B002804D00121684601F05BF900E1FB
:10E830008A4C6946A0880880E088488020898880C2
:10E840008F71102202A80C99F9F70EFDE0780128CB
:10E8500004D00697079708970997E4E7102206A8BF
:10E860000C99F9F701FDDEE7E07B002813D11123B5
:10E87000032207217E4809F45FD10546282028702D
:10E880007648C078012808D01021681CF9F705FDEA
:10E89000284609F48DD1E773CBE01022681C0C994F
:10E8A000F9F7E2FCF4E7012002F048FD0121032022
:10E8B00009F412D26F48012444841F200490674851
:10E8C0000178490601D57F21049181780522114202
:10E8D00004D0FF2204998132114304910088C005BD
:10E8E00004D5032104984902084304900821624892
:10E8F0000191029003210B2304AA00970394C902FB
:10E900005E48FAF75DFE02E079E04AE089E000281F
:10E9100046D15B4806218786FF2005905948019122
:10E920000290082305AA0097039457495748FAF71D
:10E9300047FE00287DD100F047FF002879D1022151
:10E94000032009F4C9D1B079012808D001F00CF8EE
:10E950003E484078C0076CD001F04EFB69E000F003
:10E96000DBFF66E001F032FEE77300F02DFF0028C8
:10E970005FD10221032009F4AFD1B0790128EED094
:10E9800000F0F2FF31484078C007E5D151E06878E7
:10E9900000284ED0F179481EF0713D4801F08EFC00
:10E9A00047E07179491E052906D8A72802D1307998
:10E9B000002806D100F01EFF2878A42801D0A7283F
:10E9C00037D17079042806D0062804D0082808D04A
:10E9D0000C282ED10CE02F480168002929D0B079ED
:10E9E00004E01A480169002923D00120884720E06B
:10E9F0001648016900291CD00320884719E03771A7
:10EA0000FF20F0702075607513E0207DFF2802D094
:10EA10006878002802D000F0EBFF0AE0C8079BD11D
:10EA200007E0607DFF2802D06878002804D000F05D
:10EA3000C1FF00200DB0F0BDA07D0028F9D08807EF
:10EA4000F7D5E17D144801F045FAF2E7C04E002009
:10EA5000B04D0020BF4D0020040D0000344E0020BA
:10EA60000502000048080000A08C0000190D0000FD
:10EA7000230D0000B00B0020A4410101D20B0020A7
:10EA8000680B0020FC410101011800009C0B0020D4
:10EA9000B94D0020604E0020E84D002070B50025E3
:10EAA0000C462846401C0628FCDB254E2246307EBC
:10EAB00031461A32C96906282AD203007B441B79E1
:10EAC000DB189F4424020910171E0622A01CF9F728
:10EAD0000EFC00281BD01BE0237E092001F09AF8D1
:10EAE000002814D114E0237E212001F093F800289F
:10EAF0000DD10DE0237E162001F08CF8002806D100
:10EB000006E0237E192001F085F8002800D00125B9
:10EB10000C48807D002811D17169002901D0204660
:10EB20008847002D0AD03169002901D0022088478A
:10EB300001F0E4FA217AA01C01F0CCF9002070BDAC
:10EB4000C04E0020D04D002010B50A78000A000207
:10EB500010434A78FF231B02120298431A401043C5
:10EB60008A781B02120498431A401043C9780002A5
:10EB7000000A09060843F9F76EFB002010BD10B526
:10EB8000104609F497D0002010BD0020401C062834
:10EB9000FCDB002070470000F8B51C4617460D4608
:10EBA000104609F487D0002811D1472002F062FBFB
:10EBB000064604233A460321064808F4BDD7210A35
:10EBC00001702988B288891A418008F4F1D70020A1
:10EBD000F8BD00000D470000F8B517460C46472069
:10EBE00002F048FB21780646122901D013291BD1D7
:10EBF000B06805460C351229C288018916D0062353
:10EC00000F4808F499D7698841806178017108F448
:10EC1000CFD7B068002803D008F47ED60020B060BB
:10EC20000021384609F458D00020F8BD04230548D7
:10EC300008F482D76988018061788170E7E7000075
:10EC4000094700000747000000B5084883B0026C80
:10EC5000002A08D000200090029009206B4618700E
:10EC6000684601919047002003B000BDB04D0020E0
:10EC700030B5104D83B0088828861C0A2001401941
:10EC80000A88403042822A6C0025002A07D000956D
:10EC900007206B4602951870684601919047064818
:10ECA000A1004058002801D04030C574002003B0B6
:10ECB00030BD0000B04D0020580B0020FFB581B0E2
:10ECC000002000900E46039808F4F4D7002802D0E4
:10ECD00001284CD04DE0142002F0CCFA07463188D0
:10ECE000FEF760FE05462448092D36D27C68002CCC
:10ECF0001ED02179A94203D02468002CF9D117E055
:10ED0000002C15D06379039A9B1D049908F414D73D
:10ED100005463088288000202871607968806279F3
:10ED2000A11D681DF9F7A0FA284608F441D720E094
:10ED30003D740498010A7974384602F093FA01464A
:10ED400001230E48039A08F4F7D6057008F430D76B
:10ED50000121039808F4C0D70BE00623039A049915
:10ED600008F4EAD63188018080210171DDE70220B4
:10ED70000090009805B0F0BD140C000002140000D3
:10ED8000FFB585B00E46079808F494D7002802D046
:10ED9000022009B0F0BD472002F06CFA029000207A
:10EDA000694608700898070A308803F068F900245B
:10EDB000694605468C8000281ED102981622016AF9
:10EDC0006846007803465043024610328A5A52047D
:10EDD000920F1FD10A5C401C085C1E4900021018EB
:10EDE000884217D102AA03A9184603F05BF80298DB
:10EDF0006946C05D88800224A31D1748079A0899B8
:10EE000008F49AD60746308838803D717C80002D02
:10EE100015D019E03946029802F024FA014604237D
:10EE20000E48079A08F488D6077069460978418029
:10EE300008F4BED60121079808F44ED707E0224611
:10EE400001A9781DF9F710FA384608F4B1D6002068
:10EE500009B0F0BD02290000140C000004470000B6
:10EE6000FFB58BB00C46472002F004FA0025694636
:10EE700005900D740E9804A9070A208803F0FFF886
:10EE8000060061D105981622016A6846007C50434D
:10EE9000024610328A5A5204920F3AD10A5C401C40
:10EEA000085C304900021018884232D1029503955F
:10EEB000208800F0DFF802A9002300911A4608A973
:10EEC000FAF796FB6846008C012109030840C0430D
:10EED000C004C0172146401CFEF70AFC0606360E89
:10EEE00032D168460997007C0190A57907AA694646
:10EEF00002F0D8FF6846028806A80799F9F7B4F926
:10EF000006A909980A460D5468460188019803F03D
:10EF100007F83946059802F0A5F9A1880D9A891DD0
:10EF20008BB20146104808F407D60546A288A11DF9
:10EF3000801DF9F799F92F706846007C6880A088D9
:10EF4000A880284608F434D6042308480D9A0E9960
:10EF500008F4F2D521880180867008F429D60020B3
:10EF60000FB0F0BD022900000A470000160C000097
:10EF7000F0B589B00446FAF741FB05460026154F67
:10EF80001BE006A92046FAF709FB002302AA01A903
:10EF900006A80096FAF738FB68460089B84203D104
:10EFA00069460979022911D00B49884203D1684684
:10EFB0000079022807D0641CA4B2A888A04202D815
:10EFC000E888A042DDD2002009B0F0BD204609B09B
:10EFD000F0BD00000229000003280000F7B500285A
:10EFE00045D00199002942D08668002A01D10CE061
:10EFF0003668002E3BD0316A002938D00198F9F7E5
:10F000005EF90028F4D12CE03668002E2FD0019C48
:10F01000356A002CF8D0002DF6D0AC4224D02078F0
:10F02000F9F70AF907462878F9F706F987420DD16A
:10F030002078002813D06078641C6D1CF9F7FCF868
:10F0400007462878F9F7F8F88742F1D02078F9F7E1
:10F05000F3F804462878F9F7EFF88442D4D1002E6B
:10F0600005D0306A002802D0304603B0F0BD002041
:10F0700003B0F0BDF0B589B00446FAF7BFFA054613
:10F080000026104F14E006A92046FAF787FA00235D
:10F0900002AA01A906A80096FAF7B6FA68460089FE
:10F0A000B84203D1641CA0B209B0F0BD641EA4B282
:10F0B000A888A04202D8E888A042E4D2002009B083
:10F0C000F0BD00000328000070B5164C2078002821
:10F0D00027D101210803FBF7BDFF0020FBF7B0FF9C
:10F0E0000120FBF7DBFF104D2846FAF73BFB03211D
:10F0F0002846FAF7A7FB01212846FAF767FB01210A
:10F1000021702846FAF78AFB142003F0C1FC702016
:10F1100000F00CF8702000F009F800212846FAF7FA
:10F120007DFB70BD844700200008024070B5054695
:10F13000164CFFF7C9FF2946154D2846FAF79DFAE8
:10F1400001212846FAF738FB01212846FAF772FB1D
:10F15000002807D1641E13D001212846FAF76AFB64
:10F160000028F7D001212846FAF784FA2846FAF752
:10F170005EFB044600212846FAF71EFB204670BDC0
:10F1800000212846FAF718FB024870BDA08601004E
:10F1900000080240FFFF0000F7B5042702253F4E9C
:10F1A00084B01446072A75D21000784400790018FC
:10F1B000874470030D3A3D5363003948009701902E
:10F1C00001AB0599049800F075F807B0F0BD354F14
:10F1D00001213846FAF722FB142003F059FC702075
:10F1E000FFF7A4FF7020FFF7A1FF04460021384677
:10F1F000FAF714FB2C48B442448001D12B4808E0B4
:10F200002046FAF741FA2A49F9F702FBF9F71EFD01
:10F2100000B26946888100952A4603AB0599049897
:10F2200000F048F807B0F0BDFDF7F4FA0AE06020FE
:10F23000FFF77CFFB04201D1002003E06021FAF724
:10F240004DFA80B269460881009502AB22460599C5
:10F25000049800F02FF807B0F0BD04F05BF97D21B1
:10F26000C900F8F78FFF0097019001AB224605997E
:10F27000049800F01FF807B0F0BD03F045FD0097BB
:10F28000019001AB22460599049800F013F807B0ED
:10F29000F0BDFFE7059807B0F0BD0000FFFF0000DC
:10F2A0000E0001000008024084470020FF7F00009C
:10F2B0000000204130B4029C42540546491C88B2EB
:10F2C0002C54401C002180B2002C07D95A5C2A54CF
:10F2D000401C491CC9B280B2A142F7D330BC704770
:10F2E00010B5084C82B02078002808D1064800905C
:10F2F000064801906846FEF7EBF80120207002B046
:10F3000010BD0000A0470020751D0101352A010134
:10F31000F8B50B30C608F600104D19E02068B04271
:10F3200015D3B0420BD96368871B201D0093F8F7F3
:10F330009BFFA019009B07604360286004E06068A1
:10F340002860201DF8F790FF201D2660F8BD251DC0
:10F350002C68002CE2D10020F8BD000000480020FD
:10F36000FF25F5350A4E6F00FDF7D6FB0489322CD8
:10F3700000D22C4601213046FBF74EFD7D21204670
:10F38000C90048433946F8F7FDFE03F081FBEBE77F
:10F39000000C014010B5A0230949022809D0002221
:10F3A00003280AD0042808D00B704A7000F0A2F895
:10F3B00010BD0B7080204870F8E7E0200870F4E77B
:10F3C00011400020F8B52A49202048602948012131
:10F3D000C163294905228A610021C16327490B20A5
:10F3E000086100F087F82748254A026326494163EF
:10F3F000264B8363264CC4632748264D0560274E61
:10F400004660274981602749C16027490161274932
:10F4100041612749816127490163284826494160A4
:10F42000274FC760274F07610262274A4262836203
:10F43000C46205634663254A8263254AC26326483F
:10F44000244A0260184A4260244A826001632449C7
:10F4500081632448244A41688918244A914206D28B
:10F46000234982680A63C2684A6300698863F8BDF9
:10F4700000100140C02702404025024040270240C2
:10F480000259F80040280240025B8500025A8000C1
:10F49000025D8500025F80508028024002000878EB
:10F4A000020A0800026EAC500259FC000200C800BB
:10F4B0001270131402700314026E2800C028024058
:10F4C000025D0500125B0500025B8400020A060073
:10F4D000026E2C5002C3BF00002902401200AC0093
:10F4E000125D0500104000206F2895FFAF590F00F6
:10F4F000C026024030B415481549037D154AFF2B3C
:10F5000006D1407DFF2803D113484078C0070CD0B6
:10F510001248134B04789C604078D8611148086108
:10F52000114B8B62106030BC7047104B0B61104860
:10F530004861104C8C61104D8D62C8620F480863A1
:10F5400013600F485060946030BC7047D04D00206D
:10F550000028024040280240C04E002011400020F8
:10F5600000270240127E0200127E0300027E02008B
:10F5700002C2A00012C70000027E030012C7800072
:10F5800002C2E00082B0224920480863FDF7A0FDD6
:10F5900020A0FBF779FF2AA0FBF776FF31A134A06A
:10F5A000FBF772FF3848016838A0FBF76DFF3EA1FA
:10F5B00042A0FBF769FF4AA0FBF766FFFCF7A0FD3E
:10F5C000FCF790FE01215148FBF72AFC40215048EE
:10F5D000FBF726FCFDF7A4FA01F03AF8022000241C
:10F5E0000202009023464BA101944B4803F0C6FE53
:10F5F000012000900023802248A10194484803F094
:10F60000BDFEFAF7DDFA03F01DFBFEE70080008186
:10F61000007000400A3D3D3D3D3D3D3D3D3D3D3D91
:10F620003D3D3D3D3D3D3D3D3D3D3D3D3D3D3D3D0A
:10F630003D3D3D3D3D3D3D3D3D3D3D3D3D0A0000A7
:10F64000206D636D2D6464632D626C653A20424CBD
:10F6500045202B204672656552544F53202B204382
:10F660004C490A0056312E30302E31340000000053
:10F67000204669726D776172652076657273696F75
:10F680006E2025730A00000000400020205379738B
:10F6900074656D436F7265436C6F636B203D20250D
:10F6A0006C7520487A0A000043414949432D4D4377
:10F6B0004D2D3230323630393032000020424C4548
:10F6C00020656E61626C65642C206164766572747D
:10F6D0006973696E6720617320222573220A000016
:10F6E0003D3D3D3D3D3D3D3D3D3D3D3D3D3D3D3D4A
:10F6F0003D3D3D3D3D3D3D3D3D3D3D3D3D3D3D3D3A
:10F700003D3D3D3D3D3D3D3D0A000000000C0140BA
:10F7100000080140424C450085CE00014C454400A4
:10F7200061F3000110B50124E4022046FBF764FAFE
:10F73000002805D02046FBF759FA0D490220087031
:10F74000012424032046FBF757FA00280AD020465C
:10F75000FBF74CFABFF34F8F07490648C860BFF369
:10F760004F8FFEE705484068002800D0804710BD55
:10F77000800000200400FA0500ED00E04040002079
:10F7800006480068002800D08047BFF34F8F054926
:10F790000348C860BFF34F8FFEE7000040400020E1
:10F7A0000400FA0500ED00E0064A11780A2907D2A4
:10F7B0008900891848601078401C1070012070473B
:10F7C00000207047304D002010B5084C084AE17900
:10F7D00013780020994207D288008018406880473B
:10F7E000E079401CE071012010BD0000B04D002008
:10F7F000304D0020F8B5324D05262979284680790C
:10F80000304C08290CD20A007A4412799218974495
:10F8100003080D1313191C2A052801D0FCF7E4FE78
:10F82000F8BD022808D0FDF7F5F9F8BD607B002887
:10F8300002D1E079002802D0FDF78AFAF8BDFDF781
:10F8400025FAF8BD06202871F8BD022303220721FE
:10F850001D4808F471D1A5210170E9784170072194
:10F8600029716E7128E0022303220721174808F44A
:10F8700063D10746A7203870E9787970062068714F
:10F8800000202871032008F415D2032812D0A8798B
:10F89000012804D0022802D003280BD104E0207DE7
:10F8A000002801D0032003E0A07E002802D004201D
:10F8B000A87100E0AE71384608F47AD1F8BD0000B6
:10F8C000B04D0020A04E0020A20D0000A30D0000AE
:10F8D00010B5002804D0014660220C48F8F7C4FC9B
:10F8E0000B490C48CA781C2A04D9427B002A01D152
:10F8F0001C22CA70C1781F2901D91F21C170017B48
:10F90000E22901D9E221017310BD0000604E002000
:10F91000804E0020A04E00201149012208790728BE
:10F920000CD08879002809D0012801D0052806D1FB
:10F930000C48827B002A03D002200CE08A717047B9
:10F94000027D002A01D0032005E0807E002801D03E
:10F95000042000E00520887110B5FCF745FE10BDBD
:10F96000B04D0020A04E002070B5104C0525A079A8
:10F97000062809D201007944097949188F44020206
:10F9800004040403A57170BDA5710223032207219D
:10F99000074808F4D1D0A5210170E1784170072112
:10F9A0002171657108F404D170BD0000B04D0020D4
:10F9B000A20D000010B50B4C607DFF2810D0022373
:10F9C00003220721084808F4B7D0A7210170617D00
:10F9D0004170064A00215171FF21617508F4E8D099
:10F9E00010BD0000D04D0020A30D0000B04D002040
:10F9F00010B50A4C207DFF280ED0022303220721D8
:10FA0000074808F499D0A7210170217D4170054A6B
:10FA10000021517108F4CCD010BD0000D04D002061
:10FA2000A30D0000B04D002010B5084802238078D7
:10FA3000032201020648083108F47ED0012101703A
:10FA40001321417008F4B4D010BD0000B04D002067
:10FA5000040E000010B584B0002804D001462A220C
:10FA60000E48F8F701FC0EA00FC86C460FC40B4BF4
:10FA7000002069461C180A5C247922430A54401C61
:10FA8000C0B20628F6D310220A48F8F7EDFB0A495F
:10FA90000A48F9F77DFD04B010BD0000344E002087
:10FAA000501921901F04D5624FA489AB90D0CF2369
:10FAB00000000000BF4D0020384E0020FC00002058
:10FAC0000020074B01460A01D2184032927AFF2AE1
:10FAD00001D0401CC0B2491CC9B20329F3D37047FE
:10FAE000B04D0020F8B507460B46282043430D468D
:10FAF000032207210E489B1C08F41ED0912101709F
:10FB0000002406464570002D0ED920462821484382
:10FB1000C1190022CA7180192822801CF8F7A4FBA1
:10FB2000641CE4B2AC42F0D3304608F441D0F8BDD6
:10FB3000910D0000F8B57D262025F600184B194CD4
:10FB40001949032812D00A6A01273A430A620A6A4D
:10FB50009207FCD50A6AAA430A6201281AD0022831
:10FB60001AD01E60F9F756FD2060F8BD0F480F2728
:10FB700082683F023A438260086A042210430862A6
:10FB8000086A0007FCD5086A284308623D20000186
:10FB90001E60E9E7064800E006481860E2E700005A
:10FBA0008C00002090000020001002400010014056
:10FBB000D10300005704000010B504460848042390
:10FBC0008078032201020748891D07F4B5D706494A
:10FBD0004C80012101700021418007F4E9D710BD5C
:10FBE000B04D0020010C0000F00B0020084A1178F5
:10FBF0000A290AD2C9004368891800688B604860E6
:10FC00001078401C107001207047002070470000E1
:10FC10005C4D0020FFB581B01C00064618D010785E
:10FC2000411CA14214D8032C12D3401EC5B25078F7
:10FC3000971CB04206D12A4638460299F8F757FB7E
:10FC4000002808D07A19601B801E0406240EE6D115
:10FC5000002005B0F0BD012005B0F0BDF0B50446B0
:10FC60006F4E704883B06D4FB168C1626E490163D9
:10FC7000F16A8162F16B4163B16B816331467C2231
:10FC800040313846F8F7F0FA00257D60FD607D626E
:10FC90006648B8627D64BD64FD643D666448B866CC
:10FCA00064483862644865490570032008706448F8
:10FCB000F91401600904016089140160F068614968
:10FCC0000746401E0088604B884200D01F60366E99
:10FCD000701E0088884200D05E6001200003009002
:10FCE000694601950D710820487101278F7168469A
:10FCF000FAF790FF84215548F8F7CFFA2A215448A3
:10FD0000F8F7CBFA60215348F8F7C7FA52484F4941
:10FD1000056145618561C561056245628562C562AF
:10FD2000FF264E48CE700675467500200201521817
:10FD30004032401CC0B296720328F7D32068086492
:10FD40006068486446486189C187217A454803292B
:10FD500001D8417700E0457701212020FBF77AF9AF
:10FD6000414A4249042001F017FA424940480860DC
:10FD70000A464149052001F00FFA404A4049072050
:10FD800001F00AFA40493F4808600A463F49082006
:10FD900001F002FA3E4A3F49092001F0FDF93E48D0
:10FDA00005633E48414907703D4805703D48057070
:10FDB0003D48086001203E49C00208803D494F206F
:10FDC00008703D49082008703C48072106704670BD
:10FDD0008670C170057145718571C57111483849CA
:10FDE000C1613849016238494162002002F056FC85
:10FDF0003649032007F4B4D70021032007F46CD759
:10FE0000002001F09BFA012303220721304807F468
:10FE100093D6077007F4CCD603B0F0BDC00900201C
:10FE200000800001C000002081F700010D47002084
:10FE3000B527010125F70001C6000020D8000020E9
:10FE400000E100E0FEE7000040400020B04D00204F
:10FE5000344E0020604E0020B04E0020D04D0020D7
:10FE6000F04D0020104E00208040002080800100D6
:10FE7000713E0101C0400020C0800100004100200F
:10FE800000DB0100814100204041002040DB0100F7
:10FE9000C0460020C06102000070004060000020E9
:10FEA000C9000020610000200090D0036C000020F9
:10FEB000680000206300002064000020080100208A
:10FEC000DD11010105130101A51201010443010126
:10FED000020D0000F8B5404D0646687D3F4C0F46C8
:10FEE000FF281CD02046C268002A03D003213C48CA
:10FEF00008F4E4D03A23032207213A4807F41CD639
:10FF0000A4210170697D04464170374800220178C0
:10FF100000291ED00121A170A28002701BE06D207B
:10FF2000022303220721400107F406D6A221017013
:10FF30002E49C978417007F43BD6EF7531462C48FD
:10FF4000F9F726FB0120A87560780221084360704C
:10FF5000F8BDA270A2800120E07019214901E18062
:10FF600022482181038CE381438C2382838C63822A
:10FF7000C38CA382FF23E2824133184D23836D7823
:10FF80006D070DD50525E5706181A181018CE184A6
:10FF9000418C2185818C6185C08CA085E28523867A
:10FFA00038200755204631463230F9F7F1FAE0782B
:10FFB000810703D50220FFF7EDF906E0400701D5E0
:10FFC000032000E00120FFF7E5F90A490C20487101
:10FFD000204607F4EDD5F8BDD04D0020C04E0020DE
:10FFE000030F0000A10D0000304E0020344E002011
:10FFF000E84D0020B04D0020F8B52C4E2C4D317D41
:020000040101F8
:1000000001276878FF2941D0C1073ED0B843687006
:100010002849002008703A2303220721264807F4C4
:100020008BD50446A4202070307D60702878A070A5
:1000300068788006800F20716888E080A888208119
:10004000E888E08128892082E7700120FFF7A2F983
:10005000687840070AD5E07802210843E070688894
:100060006081A888A0810320FFF794F968780007D1
:1000700003D5E0780C210843E0701049082048714E
:100080000020B075204607F493D5F8BD384368705A
:100090006D20022303220721400107F44DD5A12141
:1000A00001700749C9784170EDE70000D04D00208C
:1000B000C04E0020304E0020A10D0000B04D0020A9
:1000C000344E002010B50A4C607DFF280ED002236C
:1000D00003220721074807F42FD5A5210170617D70
:1000E0004170054A0D21517107F462D510BD000021
:1000F000D04D0020A20D0000B04D002070B50B4C7B
:10010000207DFF2811D00A4D687909280DD00223DF
:1001100003220721074807F40FD5A5210170217D8F
:1001200041700921697107F443D570BDD04D00209D
:10013000B04D0020A20D000010B504464088A188F3
:100140000246491C19234A43DB019A420FDC062868
:100150000DD3228890420AD3E2887D23DB009A42A5
:1001600005D84B00C9184843D100884201DD002062
:1001700010BD0D480E238078032201020B48083180
:1001800007F4DAD4092101702188418061888180D7
:10019000A188C180E188018100214181491E8181BE
:1001A00007F406D5012010BDB04D00200E0E000052
:1001B00010B5084A084B906901888478994206D1A5
:1001C000917CA14204D20024FAF7FAFE00E0002458
:1001D000204610BD104D0020341200000B4610B513
:1001E00004493A228969504341181846091DF8F715
:1001F0003BF810BD104D002010B590B004463C21D6
:100200006846F8F74AF8FFF7D3FF401EC0B26946C8
:10021000FFF7E4FF08A8807CA0710CA920460331F9
:10022000F9F7B6F910B010BD10B590B004463C21F6
:100230006846F8F732F8FFF7BBFF401EC0B26946C8
:10024000FFF7CCFF08A8007CA0710AA92046023164
:10025000F9F79EF910B010BD10B590B004463C21DE
:100260006846F8F71AF8FFF7A3FF401EC0B26946C8
:10027000FFF7B4FF0AA920460231F9F789F908A867
:10028000007CA071204606A9102208300231F7F741
:10029000EBFF0848C17820461830012904D010210E
:1002A000F7F7FBFF10B010BD10220349F7F7DCFF92
:1002B00010B010BD344E0020BF4D002070B590B07E
:1002C0000D460646FFF774FF002D23D0854221D846
:1002D000182303220721104807F42ED404461720C0
:1002E0002070012060703146A01CF9F751F93C21C3
:1002F0006846F7F7D2FF6D1EE8B26946FFF76EFF5A
:10030000204606A9102208300231F7F7ADFF20463B
:1003100007F44ED410B070BD140D0000F3B58FB0CB
:100320000C463C216846F7F7B8FFFFF741FF012C68
:100330001AD0002816D0154D0AAE0236441EE0B27F
:100340003A22A969504341186846091DF7F78CFF06
:10035000062231460F98F7F7CAFF00280DD0200675
:10036000000EEBD111B0F0BD0949421ECA71014621
:100370000F98FFF7A3FF11B0F0BD06A910220548A2
:100380000231F7F771FF11B0F0BD0000104D0020F1
:10039000B04D0020CF4D002070B5284C82B02068B1
:1003A0008003FCD5264D687FFFF7C4FB606A606A56
:1003B000012630436062606AB04360622148C08FAA
:1003C0000A2811D9E16932071143E1611E494A68DF
:1003D00032434A601E491D4A0A6003224A6088600F
:1003E0001C4808601C48086068461BF437D11B494C
:1003F00000980860687FFF252D02032811D000F0C7
:1004000027F9206BA8432063206B3F214902084352
:100410002063206B3043206301220321104807F43E
:100420004DD610480168A94301600F490868FF22B2
:1004300012049043086002B070BD0000001002403A
:10044000104E0020F04D0020401002405555000095
:1004500000300040AAAA0000CCCC00004840002098
:10046000010F000000E400E008E400E0F0B5D7B0C0
:1004700054A81BF4F3D04A490024886AC96A5499E5
:100480000122411A09010909D206914204D954995D
:10049000081A000100094142424E40290CDC7088D4
:1004A000002809D0401E7080142203213E4807F422
:1004B00005D6002057B0F0BD3C48FF2156902931A9
:1004C0006846F7F7EAFE707CB569002832D0FFF77E
:1004D0006FFE69468870B17C6F4688420BD23A2124
:1004E00048430246291D381DF7F7BEFE6946887845
:1004F000401C887008E03A21401E484302462946C5
:100500003E31381DF7F7B0FE694688783A214843F6
:10051000C0190A4636385699F7F7A6FE24486946A8
:100520000880B069FAF74CFDFF2227326946B069AE
:10053000FAF774FDFF20F53070804A944B944C9488
:100540004D944E944F945094519452941748539410
:10055000418D40AA1185818D5185C08D9085154CA6
:1005600048AA257C9573102213494CA8F7F77CFE06
:100570001248C078012804D11022114950A8F7F779
:1005800073FE01260F48002DC67306D1A07C0028FB
:1005900003D001214AA8FFF7A5FA0B48067088E7A7
:1005A000C0800240104D0020040F0000D44C0020F9
:1005B00034120000F44C0020EE4C0020344E002099
:1005C000BF4D0020D04D0020304E00200248007862
:1005D000002800D001207047104D0020014800790C
:1005E00070470000104D002070B517493CC80E46FA
:1005F00084B040363CC64368026880684B65134C43
:100600000A658865607C002818D0002569460D724F
:10061000FAF7E8FCFFF7CCFD69460872E1690126AC
:10062000002906D068460095067002A80190684629
:1006300088476846007A002802D0267004B070BD52
:10064000257004B070BD0000D44C0020104D002077
:1006500004490868401C0860012801D00120704747
:10066000002070472440002003490868002802D079
:10067000401E08600120704724400020F8B50C4659
:100680002849294B4118294F294A0026069D00294F
:1006900008D0012922D0274940180A282FD3012049
:1006A0002870F8BD20780A2838D2214980000958DE
:1006B000214A914203D11E490E501E502EE0B942EC
:1006C0002CD10322082311461C4807F435D2217887
:1006D00001706168416007F46BD21FE020780A283E
:1006E0001CD280001158B94218D1195811502078E5
:1006F000134962684018032107F4E0D40EE0C0B249
:100700000A280BD284001159002907D0B94205D01C
:10071000094FB94202D016511E5188472E70002051
:10072000F8BD0000FBF0FFFFAC4C0020CB2801011E
:10073000844C0020F9F0FFFFC9280101060F0000DA
:10074000070F0000F7B5534F3878002809D0042A66
:1007500009D2012211217B69009800F075F903B0DC
:10076000F0BD002314E00C784E7820468C783602D9
:10077000CB783043240420431B061843CB78000277
:10078000000A1B0618437B690D1D141F984206D0F2
:1007900002221121009800F057F903B0F0BDB868AB
:1007A0001E19864203D90322112100986DE07E6153
:1007B000F869B0420FD2F96978684018FAF700FC7E
:1007C000002801D0052207E00120F969000308187C
:1007D000F861B042EFD30022002A3CD1B86A002869
:1007E00022D02D49042808D2002C1BD02B780B5482
:1007F000401C641E6D1CB862F4E73E46042811D10B
:10080000B1697068244B401804221946FAF706FCB7
:10081000002801D0052203E0B069001D0022B0616C
:100820000020B062002A16D1042C1DD3BA69786862
:10083000A608B600801829463246FAF7EFFB0028D2
:1008400001D0052203E0B86980190022B861AD1912
:10085000A41B002A08D011217B69009800F0F4F84D
:10086000FCF7C0F803B0F0BD002C05D022462946A5
:100870000948F7F7F9FCBC62BB693A6A0098190BA2
:100880009142EFD939620022112100F0DDF803B066
:10089000F0BD0000584700207C470020F7B5634DAD
:1008A0008CB028780B46002809D0042A09D00122F0
:1008B00012216B690C9800F0C7F80FB0F0BD00234F
:1008C00013E01A78D97810465A78090612021043B4
:1008D0009A781204104308430402D878240A0006C8
:1008E00004436B69A868834206D0022212210C9847
:1008F00000F0AAF80FB0F0BDA86A0026002815D0B5
:10090000042806D24A4AFF211154401CA862042838
:10091000FAD3AB69686846490422C018FAF77EFB2F
:10092000002867D1A869AE62001DA861A96868683F
:10093000FCF7C4FEA04202D1E968884209D0042233
:1009400012216B690C9800F07FF8FCF74BF80FB0A0
:10095000F0BD384C6F460FCC0FC70FCC0FC7A26845
:10096000616820680A920890334F0098203C0991F2
:10097000B84206D128212046FCF7A0FE0A998842F9
:100980000AD000960196029603960496059606965E
:100990000796089609960A960097284A6968914230
:1009A00001D1012000E0022001909142684601D16E
:1009B000083000E018300160A9684160E968816092
:1009C0002969C16028216846FCF778FE0A90204614
:1009D000FAF7F6FA00280DD12C2269462046FAF7DC
:1009E0001DFB002806D12C2221466846F7F77FFC24
:1009F000002809D0052212216B690C9800F024F818
:100A0000FBF7F0FF0FB0F0BD00221221AB680C988D
:100A100000F01AF8C82002F03BF8BFF34F8F0949E5
:100A20000748C860BFF34F8FFEE70000584700201B
:100A30007C4700200040000111C011CA0080000165
:100A40000400FA0500ED00E010B582B06C4621709C
:100A50006270A370190AE170190C2171190E61718D
:100A6000014606236A461F20FBF732FD02B010BD87
:100A700070B5FEF735FCFCF7EFFC04002FD01A4DE3
:100A80002889F8F7C7F802460B4618A12046FCF75C
:100A900097FCE868F8F7BEF802460B4614A120461A
:100AA000FCF78EFC13480078F8F7B4F802460B46C2
:100AB00011A12046FCF784FC2046FCF7DDFD05462D
:100AC0002046FCF7D5FC002D09D02846FCF7F4FEA3
:100AD0000BA0FCF7F1FE2846FCF7D6FD70BD09A07F
:100AE000FCF7EAFE70BD0000A45C00206C656400A9
:100AF00070776D008847002076616C6964000000A3
:100B00000D0A00006A736F6E3A20616C6C6F63208F
:100B10006661696C0D0A000070B5134C01256078A0
:100B2000002802D1FAF75EFA657010483021FCF710
:100B3000C5FD0E490E4E08633046FAF741FA00280B
:100B40000DD1342209493046FAF768FA002806D157
:100B5000342231460548F7F7CAFB002801D00120AE
:100B600070BD2570002070BD88470020A45C002067
:100B700000600001F3B583B0049800210668806826
:100B8000009137187D1C305C2C4622287ED10498B9
:100B9000406807E05C2A04D15B1C834277D2491C81
:100BA000641C641CA31B834202D22278222AF1D146
:100BB000A21B82426BD22078222868D1E01B401A07
:100BC0000499401C09698847009000285ED0A5421E
:100BD00070D229785C2903D00170401C6D1CD8E0CC
:100BE0000223611B012952DB6A78662A15D008DCD2
:100BF000222A22D02F2A20D05C2A1ED0622A46D157
:100C000008E06E2A0DD0722A0FD0742A11D0752AEE
:100C10003DD115E00821017010E00C210170401C4D
:100C2000B6E00A210170401CB2E00D210170401CA9
:100C3000AEE009210170401CAAE00270401CA7E050
:100C40000022944606296FDBAF1C1346F95C0E4662
:100C5000303E092E02D8303A8A180BE00E46413E4B
:100C6000052E01D8373A04E00E46613E052E1FD806
:100C7000573A8A18032B00D212015B1C042BE5D3D0
:100C800037218902531A55498B4201E09CE094E0D8
:100C90007BD91B23DB02D31A8B423FD80C23A91D1F
:100CA0009E46631A062B70DB0B785C2B6DD102E03D
:100CB0000022E5E770E04B78752B66D1891C019125
:100CC00000210E46019B9B5D1F46303F092F02D835
:100CD000303959180BE01F46413F052F01D83739ED
:100CE00004E01F46613F052F16D857395918032EC7
:100CF00000D20901761C042EE4D337239B02CE1ABE
:100D000001239B029E4240D292058905120B890D58
:100D10000A439901521803E00021EEE706218E46AE
:100D2000802A02D2012315E02FE00121C9028A4264
:100D300003D20223C0218C460CE0012109048A421F
:100D400002D20323E02104E025498A421DD804236E
:100D5000F0218C46591E0906090E0AD01646802736
:100D60003E43BF273E404654491E92090906090EDC
:100D7000F4D1012B03D961460A43027002E0510607
:100D8000490E0170C018734600E00023002B14D0F8
:100D9000ED18A54200D21CE7002101700398102134
:100DA000C160039900980861049804990068201AAA
:100DB000401C8860012005B0F0BD0098002803D0D9
:100DC0000498416900988847002D04D00498006871
:100DD000291A04988160002005B0F0BDFF030000CF
:100DE000FFFF1000F0B591B00C0006467ED02168E0
:100DF00000297BD0A0686368021D9A4206D80818B3
:100E00000422DBA1F7F789FA002833D0A0686268D2
:100E1000411D914207D8216805220818D6A1F7F78D
:100E20007CFA00282ED0A0686268011D914207D884
:100E3000216804220818D2A1F7F76FFA002829D0F8
:100E40006268A168914203D22068405C22282BD0BE
:100E500091427AD22068405C2D2802D0303809288F
:100E600073D800200146109020682E22002807D059
:100E70006B464DE00420F060A068001DA0600120DA
:100E800011B0F0BD0120F060A068401DA0600120FD
:100E900011B0F0BD0220F06001207061A068001D5B
:100EA000A060012011B0F0BD21463046FFF762FE80
:100EB00011B0F0BD25682818085C342820D00DDC5E
:100EC00005462B3D092D28D22F007F443F79FF197D
:100ED000BF441623161823161616160038280FD0EE
:100EE00008DC35280CD036280AD000E074E037281A
:100EF00013D105E0392803D0452801D065280CD14D
:100F0000585400E05A54491C3F2906D2002C04D002
:100F1000A06867684518BD42CCD30020585410A97A
:100F2000184601F0C3FC0F460546109968468842F2
:100F300052D0F761944A954B28463946B561F7F788
:100F40000BFF03D8924870610FE019E00022914B2B
:100F500028463946F7F7ECFE02D80120C00703E027
:100F600028463946F7F78CFE70610820F060109A29
:100F7000A1686846101A0818A060012011B0F0BDE1
:100F80007D20C000914203D223685B5C5B2B06D0BE
:100F9000914279D22268515C7B2967D074E00027A6
:100FA000E1683D4681426FD2491CE1602168A0683A
:100FB000095C5B2968D1401CA0602046FCF7E2F97F
:100FC0006168A068884203D22268125C5D2A38D02A
:100FD000884202D3401EA06056E0401EA06020461A
:100FE00010300090FCF7AEFA002839D0002F23D043
:100FF000286045600546A068401CA0602046FCF7BC
:10100000C1F921462846FFF7EDFE00282AD02046E8
:10101000FCF7B8F9002C25D06168A068884203D29B
:101020002168095C2C290AD0626890421AD2216892
:10103000085C5D2816D104E007463D46DBE70098D2
:10104000D0E7E068401EE060002F00D07D602020E7
:10105000B760F060A068401CA060012011B0F0BD36
:10106000002F11D03846FCF703FA0DE00027E168A5
:101070003D46814208D2491CE1606168A06888420F
:1010800002D2115C7B2902D0002011B0F0BD401CBF
:10109000A0602046FCF776F96168A068884203D218
:1010A0002268125C7D2A4CD0884293D2401EA060F8
:1010B000204610300090FCF745FA002855D0002F4C
:1010C0004ED0286045600546002CCBD0A0686168F2
:1010D000401C8842C6D2A0602046FCF753F9214646
:1010E0002846FFF747FD0028BCD02046FCF74AF908
:1010F00028692862002028616168A0688842B1D20E
:101100002168095C3A29ADD1401CA0602046FCF75B
:1011100039F921462846FFF765FE0028A2D020466F
:10112000FCF730F96168A068884203D22168095C45
:101130002C2918D06268904294D22168085C7D28DE
:1011400090D1E068401EE060002F00D07D6040201C
:10115000B760F060A068401CA060012011B0F0BD35
:1011600007463D46B0E70098A5E7002F8CD079E709
:101170006E756C6C0000000066616C7365000000A9
:1011800074727565000000000000C0FFFFFFDF41C2
:10119000FFFFFF7F0000E0C1102819D230B40D4CD2
:1011A00083001B199D6989032D0B2D03090D0D4328
:1011B0009D619969084D920992052940920A11434F
:1011C00099610122616982401143616130BC7047BD
:1011D0007047000000200240FF0FC0FFF3B5054636
:1011E00081B00026408800F003F901000AD01C4FAE
:1011F0006A88002014234343DB195B8A934203D19E
:1012000042262AE0402628E0401CC0B20A28F1D33A
:10121000002E22D1002414206043C019408AFF28E8
:1012200006D0641CE4B20A2CF5D30A2C14D014E0C6
:1012300028460830009014206043C0190E686B786F
:10124000AA880746A91DB0470600EED168887882B3
:101250000298398A0180E8E74B26304603B0F0BD9A
:10126000684B002002885004400CD20B01D00902C8
:101270000843704710B40024094A214614234B4305
:101280009B185B8A834204D1142041438818C468A8
:1012900003E0491CC9B20A29F0D3204610BC7047AC
:1012A000684B002030B4FF23040AC5B20A4900206D
:1012B000142242435218128AAA4204D114225043E3
:1012C0004018438A03E0401CC0B20A28F0D3200231
:1012D00030BC184370470000684B0020084A117862
:1012E0000A290AD2C9004368891800688B604860DF
:1012F0001078401C107001207047002070470000DB
:10130000304C002030B4FF23040AC5B20A49002043
:10131000142242435218528AAA4204D11422504342
:101320004018038A03E0401CC0B20A28F0D3200210
:1013300030BC184370470000684B0020F1B582B004
:101340000299294E0020002900D130700025029812
:10135000002804D0012834D002283ED10FE02946CD
:1013600014225143214A284609308C182082C0B2E9
:1013700006F410D5207C214606F4F2D42DE0284650
:1013800014214843194900234718B87C009030784D
:101390001C4600280DD9E0008019828800998A42F5
:1013A00002D1806880470346641C3078E4B2A042D2
:1013B000F1D8002B02D0596838468847387C06F4AB
:1013C0000DD51422094B6A430021D018FF24C160B7
:1013D000448299504160018141816D1CEDB20A2D1A
:1013E000B5D303B0F0BD0000304C0020684B0020A6
:1013F00070B50146094DCEB2002029780446002977
:101400000BD9E10049198A88B24201D18868804726
:10141000641C2978E4B2A142F3D870BD304C00209E
:10142000F7B500248AB000940194029403940E4608
:1014300004940594069407940894FF2701371168D3
:10144000154638468847059601970090AA6869684E
:101450002868069000980892079100283CD06946B9
:101460000A9800F0CDF8002830D00098002806D067
:1014700002994018F6F71CFF029940180290AA68DA
:10148000002A07D002990098491C904706001DD0F9
:10149000009418E002982968401C8847060015D07F
:1014A00002980199401C814201D20A4601E0029A49
:1014B000521C30460099F6F7D7FE029834546968FA
:1014C00000988847009430460DB0F0BD0098002881
:1014D00002D069688847009400200DB0F0BD00007C
:1014E000F8B500240A460546002910D0002D10D07A
:1014F00001460078002826D008780C283BD015DC5F
:10150000082838D0092836D00A2815D133E0002021
:10151000F8BD03211046FCF7FDFB0028F8D022217E
:1015200001704170002181700120F8BD0D2822D08A
:10153000222820D05C281ED0202800D2641D4878A4
:10154000491C0028D8D1481B0719F91C1046FCF784
:10155000E1FB061EE9D0002C0FD022203070287845
:10156000741C002834D0C0B21F2813D9222811D0EF
:101570005C2837D10EE0641CE1E7222434703A463F
:101580002946701CF6F770FEF01944700021817036
:101590000120F8BD5C2020702A78641C0C2A23D01E
:1015A00006DC082A1DD0092A24D00A2A06D11DE00B
:1015B0000D2A1DD0222A12D05C2A13D00EA120465B
:1015C000F9F772FF241D6878641C6D1C0028CAD1CD
:1015D0002221F0194170002181700120F8BD2220E4
:1015E00000E062202070EEE76620FBE76E20F9E75E
:1015F0007220F7E77420F5E7752530347800000095
:10160000002801D0002901D100207047F0B505461F
:10161000007B8BB00C4610287ED008DC012819D046
:10162000022821D0042809D0082876D128E02028D3
:1016300074D0402873D080287DD19BE005212046BE
:10164000FCF768FB002803D0DCA1F7F7E9FF0120D5
:101650000BB0F0BD06212046FCF75CFB0028F7D05C
:10166000D8A1F7F795FF08E005212046FCF752FBCB
:101670000028EDD0D5A1F7F7D3FF01200BB0F0BDC6
:1016800007910024AF69EE6900942E200194039421
:1016900004940594029406940894314609940A909F
:1016A000002F01D0012000E0002001434800C9497B
:1016B0004008081AC00F14D1012170004905C84222
:1016C00001D1002F0DD06869F7F790FA3A463346FA
:1016D000F7F72EFB0BD1C0A168466A69F9F7E4FE63
:1016E00026E0BEA16846F9F7DFFE054621E03A464E
:1016F0003346BCA16846F9F7D7FE054608AABBA148
:101700006846F6F719FE01280CD13A463346099986
:101710000898FCF7E3F803E03EE00CE041E094E0D9
:10172000002806D13A463346B1A16846F9F7BCFE17
:1017300005461A2D02D300200BB0F0BD691C079896
:10174000FCF7E8FA0028F7D0002D0BD92E236A46C3
:10175000115D0A9EB14201D1035500E00155641CA0
:10176000AC42F5D3002101550798806841190798CC
:10177000816082E728690028DED0F6F799FD401CD9
:10178000064601462046FCF7C5FA0028D4D032466A
:101790002969F6F769FD70E72869FFF7A1FE0BB02C
:1017A000F0BDAD6801212046FCF7B4FA0028F6D060
:1017B0005B210170A068401CA060E068401CE060F4
:1017C000002D34D0002621462846FFF719FF0028B7
:1017D00013D0002C09D02068002806D0A16840183A
:1017E000F6F766FDA1684118A160286800281BD0A3
:1017F0006069002804D0022703E030460BB0F0BD3A
:101800000127791C2046FCF785FA0028F5D02C2109
:1018100001706169401C002902D020210170401C28
:101820000670A068C019A0602D68002DCBD10221E0
:101830002046FCF76FFA0028E0D05D2101700021FE
:101840004170E068401EE06017E76069AD680028FD
:1018500001D0022700E00127791C2046FCF75AFA44
:101860000028CBD07B210170E168401C491CE1605D
:1018700062690A21002A00D00170A068C019A06026
:10188000002D78D000276069002814D02046E16838
:10189000FCF740FA002825D0E2680021002A06D98A
:1018A00009220270E368401C491C8B42F9D8E168A8
:1018B000A0684018A0602146286AFFF711FE0028A2
:1018C00010D0002C09D02068002806D0A16840184C
:1018D000F6F7EEFCA1684118A1606069002804D009
:1018E000022603E038460BB0F0BD01263146204603
:1018F000FCF710FA0028F5D03A2101706169401C0C
:10190000002901D009210170A06821468019A0603A
:101910002846FFF775FE0028E4D0002C09D0206887
:10192000002806D0A1684018F6F7C2FCA16841184B
:10193000A1606069002800D001202968002900D03A
:1019400001214618711C2046FCF7E4F90028C9D093
:101950002968002902D02C210170401C61690029EE
:1019600002D00A210170401C0770A0688019A06095
:101970002D68002D87D16069002802D0E168491CDC
:1019800000E002212046FCF7C5F90028ABD06169D0
:1019900000290BD0E2680021012A07D00922027039
:1019A000E368401C491C5B1E8B42F8D87D21017006
:1019B00000214170E068401EE0605EE66E756C6C70
:1019C0000000000066616C7365000000747275654C
:1019D000000000000000F07F256400006E756C6C54
:1019E0000000000025312E3135670000256C6700AE
:1019F00025312E313767000070B505460078002884
:101A000013D00A4E2846F6F753FC84B20D2C00D9A9
:101A10000D2471782346481C70702A460220FAF77C
:101A200057FD2D1928780028ECD170BD4C470020B7
:101A3000F8B5069E1F46182E01D9182500E0354638
:101A400013460A4601460CA00096F9F71DFD002436
:101A5000002D07D9395D11A0F9F716FD641CA4B259
:101A6000AC42F7D3AE4202D90EA0F9F70DFD0FA09C
:101A7000F9F70AFDF8BD00005B424C452025735D77
:101A800020747970653D3078253032582073657147
:101A90003D2575206C656E3D257500002025303292
:101AA00058000000202E2E2E000000000D0A00001D
:101AB000F8B5134E0F46756904463068001D00F0F6
:101AC00005FF601C07D1002F05D031680D48091DA6
:101AD00000F089FFF8BD30682C1944603168AC42D1
:101AE00004D2B068091D00F065FFF8BD7068091DDB
:101AF00000F060FF306B8442F7D23463F8BD000021
:101B0000A4470020B45D0020F8B5856B1646044656
:101B10000027026C002A11D0002E19D0E068F6F7D9
:101B2000A3FB216CE068401AE0602268904202D278
:101B30006068401AE060022E17D019E02068002883
:101B400016D1606801F056FD0746002060600FE086
:101B5000A068F6F789FB216CA0684018A060616856
:101B6000884205D32068A06002E0002D00D06D1EE1
:101B70006D1CA5633846F8BD114D124E124FE86832
:101B8000002817D000F03CFFF068C468201D00F06A
:101B90009DFE2869401E2861E868401EE86000F04C
:101BA0003BFF206B00F046FF204600F043FFE86853
:101BB0000028E7D138680128E1D900F05DFFDEE7B1
:101BC000A4470020A05D0020D85C002030B412495A
:101BD00000E011460A688242FBD34B685C188442DD
:101BE00003D1406818184860084643681C1894429E
:101BF0000CD10A4C2468A24206D052689A1842605E
:101C00000A681268026002E0046000E0026081423B
:101C100000D0086030BC7047F0470020E04700204B
:101C2000F7B582B0039800260068002859D00398C1
:101C3000416802464968083241600092914201D1F0
:101C4000496841604068C0680190039841684968EC
:101C50004160009A914201D149684160CF682420D7
:101C600002997043441804983D46002F01D11E4943
:101C70000D682560294634316160E96A2161296B6C
:101C8000E161696CA1600023E96CA36161610528D1
:101C900013D015490A68954201D1237311E02073CE
:101CA00003280ED1886B401C8863A86A002801D0E5
:101CB0000220207301F040FD03E02846FBF7FAFF05
:101CC0002073286B00210278A52A04D14278401C99
:101CD000491CA52AFAD0880820840198761C8742DE
:101CE000B3D1304605B0F0BDA447002003480068DA
:101CF000401C72B600D0FEE7FEE70000F847002067
:101D0000F8B5054600F07CFE2E46403605243457D3
:101D1000002C0FDD2F462437686A00280AD0384689
:101D200001F0D8FC002801D000F03AFF641E64B234
:101D3000002CF1DC0027FF43777100F06DFE00F00E
:101D40005FFE04243457002C10DD2846103000902C
:101D5000286900280AD0009801F0BCFC002801D0B6
:101D600000F01EFF641E64B2002CF1DC377100F03D
:101D700053FEF8BDF8B50446002500F08BFF374E42
:101D800000273068364A002801D0F0681BE00521A2
:101D900034480903430705D0C01DC008314BC000BB
:101DA000C31AC91A41180839C908C9005760106018
:101DB00031604F600B1A0F6043600160B360012017
:101DC000C0077360F06004423FD1002C3DD0204634
:101DD0000830410708D04107490F0823591A08184D
:101DE000410701D072B6FEE700282ED07168884204
:101DF0002BD81B49146801E02146144662688242D0
:101E000002D22268002AF7D1326894421DD00D68B0
:101E100022680A60616808350A1A102A09D921184F
:101E20004B0701D072B6FEE74A6060600846FFF7D4
:101E3000CDFE61687068401A7060B268904200D24E
:101E4000B060F06827600143616001F075FC6807CD
:101E500001D072B6FEE72846F8BD0000E04700203A
:101E6000F0470020C85D002004490868002803D01E
:101E70000868026D521C026508687047A44700207C
:101E800010B40124031F24061C601B1F1960191FB6
:101E9000034B0B6014390A6010BC403870470000D7
:101EA000ED1C010170B5064614460D464720FFF7AC
:101EB000E1F90369002B0DD01879B04207D15879A8
:101EC0002880981D2060002B04D0002070BD1B6866
:101ED000002BF1D10020288020600A2070BD000076
:101EE00070B516460C46104605F4E4D6002813D10A
:101EF0004720FFF7BFF90546062332461946074833
:101F000005F41AD6A988628889180180A1884180C1
:101F1000A179017105F44CD6002070BD180C0000A9
:101F2000F7B506460D464720FFF7A4F904690746B2
:101F3000002C14D02079B0420BD16079A8420CD08B
:101F4000384621461030F7F747FB204605F4E4D425
:101F500005E02468002CEDD101E0002C0AD12846D0
:101F60000121083005F462D5044601463846103098
:101F7000F7F738FB267165712A46A01D0299F6F71E
:101F800073F9002003B0F0BDF8B5C5680124287FBF
:101F90000F4601281ADD0E4E2046162250430246F7
:101FA000296A10328A5A5204920F0BD10A5C401CE3
:101FB000085C00021018B04204D1E1B20022384699
:101FC00000F03EF9287F641CA042E5DCF8BD00006B
:101FD00002290000F8B5C5680124287F0F460128B2
:101FE0001ADD0E4E2046162250430246296A103250
:101FF0008A5A5204920F0BD10A5C401C085C000202
:102000001018B04204D1E1B20022384600F018F9AD
:10201000287F641CA042E5DCF8BD00000229000016
:1020200070B5C46805462069002803D00020002848
:1020300002D00EE00120FAE7264610363046F7F7C8
:10204000B9FA05F469D42069002808D000210029D4
:10205000F4D00020E860204605F45ED470BD012174
:10206000F5E710B504464720FFF704F9827900210F
:10207000A24202D98088001981B2084610BD70B50D
:1020800004460D464720FFF7F5F801468088802278
:10209000A04206D889794118A14202D9201A287095
:1020A0000022104670BDFFB585B00E9D064629780A
:1020B00001208840401E049018460E210840328AB4
:1020C00069681F46403001920023039000930291FB
:1020D0002B7804AAA9680698F7F7A8FA00900028B8
:1020E0002AD10121282005F4A1D40446AA686968F0
:1020F000286862622162E061F46006980188A1802C
:10210000217FA171F80701D00120C003079908437E
:102110002080308A608047207082304600F0AAF824
:1021200020461030F7F752FA217F206A00F008F8B5
:10213000308A002105F4D0D5009809B0F0BD000028
:10214000F3B583B00020019004980125012845DDF6
:102150001621039A69438818028A5204920F39D1D2
:10216000039A4078515C000209181D48814231D120
:1021700001A80290EFB204264720FFF77BF80090F9
:102180000469002C14D02079B8420BD16079B04298
:102190000CD0009821461030F7F71EFA204605F4BF
:1021A000BBD305E02468002CEDD101E0002C0AD15E
:1021B00030460121083005F439D404460146009820
:1021C0001030F7F70FFA277166713246A01D029999
:1021D000F6F74AF804986D1C8542B9DB05B0F0BDEE
:1021E0000229000000487047E83D010170B506462D
:1021F00010480D46007800281AD04720FFF782F8D3
:10220000A91D8BB2014603220B4805F495D4044660
:102210000A482A468078207001206070052060807E
:10222000A5803146A01DF6F71FF8204605F4C0D45E
:1022300070BD00003747002006470000B04D002069
:1022400070B584B00E461446054601AA694630466C
:10225000FFF728FE6846028802A80199F6F704F8FD
:1022600002A844550246684601883046FFF758FEEA
:1022700004B070BD10B504464720FEF7FBFF0449CB
:10228000216009216181183060600120208110BD2A
:10229000F83D0101FFB583B00C464720FEF7EAFF89
:1022A0000546808861882678401887B2059805F42D
:1022B00001D5012807D03846FCF75AFE6946FFF7DA
:1022C000DEFE002802D0022007B0F0BD01210598F3
:1022D00005F402D50C3C0020AC60287368460078F9
:1022E000687301AA02A9FFF7DDFDA86801990446F9
:1022F000895D0C34890720D5A188C28808318BB24A
:102300003102C1200001891D05F416D406461320B0
:102310003070A88861884018B080A088F08030466E
:10232000A288A11D0830F5F79FFF304605F440D480
:102330000121059805F4D0D401E005F4EDD2012087
:1023400007B0F0BD10B5FAF7A5FD002010BDFFB530
:1023500083B00C464720FEF78DFF054680886188D4
:102360002678401887B2059805F4A4D4012807D030
:102370003846FCF7FDFD6946FFF781FE002802D0D4
:10238000022007B0F0BD0C3CAC602E7368460078AC
:10239000687301AA02A9FFF785FDA86801990446A0
:1023A000895D0C34890720D0A188C28808318BB29E
:1023B0003102C1200001891D05F4BED3064612205A
:1023C0003070A88861884018B080A088F0803046BE
:1023D000A288A11D0830F5F747FF304605F4E8D381
:1023E0000121059805F478D401E005F495D2012087
:1023F00007B0F0BD10B50C464720FEF73BFF8088C4
:102400006188A31D401880B2A1880022FAF7DAFC87
:10241000002010BDF8B5488800900C468E88F9F76A
:102420006BFF00281DD0182E01D9182700E0374671
:10243000324623A00099F9F727F80025002F08D984
:102440006019817927A0F9F71FF86D1CADB2BD4264
:10245000F6D3BE4202D925A0F9F716F825A0F9F760
:1024600013F8009802281FD0062802D0082824D18B
:102470001FE0022E21D1E0881F49012802D0002848
:1024800008D01AE001200870F9F736FF002814D0B0
:102490001AA006E000200870F9F72EFF00280CD0E3
:1024A0001CA0F8F7F1FF08E0A188A01DF9F740FF94
:1024B00003E0A188A01DF9F77FFE0020F8BD000011
:1024C0005B424C455D20777269746520696E643AA1
:1024D000206174745F6964783D2575206C656E3D7C
:1024E000257500002025303258000000202E2E2EA9
:1024F000000000000D0A0000374700205B424C45F9
:102500005D206E6F7469667920656E61626C6564CA
:102510000D0A00005B424C455D206E6F7469667960
:102520002064697361626C65640D0A00FFB581B057
:1025300000276846078048881C460D46082823D097
:102540000A2825D005206946088014A66846008818
:102550002146083083B21348039A05F4EDD28771FF
:1025600029780446017068460288A28069886180E3
:10257000002A03D03146E01DF5F776FE204605F42B
:1025800017D3002005B0F0BD6846F9F78BFE02E0D6
:102590006846FAF79DF90646D8E700004E53494EC3
:1025A000470000000547000070B516460C4610466F
:1025B00005F480D3012818D1A1791A48002916D032
:1025C0002178062309023246891D05F4B5D2054655
:1025D000A078FFF746FD288080202871284605F462
:1025E000E7D20021304605F477D3002070BDA188E2
:1025F0003246891D8BB221780902891D05F49CD2CF
:102600000546A078FFF72DFD288000202871A088BE
:102610006880A288E11D681DF5F726FE284605F4AE
:10262000C7D2DEE7140C0000F3B583B005001AD062
:1026300028680190284680380290C76F04983E1F92
:10264000864200D906462846F8F774FF04460091F2
:10265000324629460498FCF75BFE0199002806D013
:10266000016005B0F0BD0498F8F796FFF9E729601E
:102670000299002CCF670AD021686218291F8A426C
:1026800002D9291B091F216000996160E9E7024A0C
:1026900000991160E5E700000048002010B5012412
:1026A00000206407206005F49DD12E4802882E4842
:1026B0000168002005F422D22C4802882C480168C9
:1026C000012005F41BD22B48008882B22A480168F9
:1026D000022005F413D22948008882B228480168F4
:1026E000032005F40BD22748416AF02211434162CE
:1026F000254818F4F5D1264824490160254941614F
:10270000254981602549C160254981612549C1610B
:10271000264925488863FCF755FE2068C0B2F6F7C5
:102720008BFF23480078002806D0002018F41ED51F
:1027300001460020F6F786FF2068C0B2F6F788FF52
:10274000F6F78CFF2068C0B218F49CD22068C0B2A3
:1027500018F4A6D22068C0B218F464D40120206016
:1027600010BD00001C0100201801002024010020E1
:102770002001002034010020300100202C01002025
:102780002801002040250240740200205002500021
:102790008080024000080F0058086A0042050000CF
:1027A0000F0505060F000F034000D00040800240D7
:1027B00062000020F0B5314C83B0E06980075AD543
:1027C00002202062A56B082018F474D5012018F4AB
:1027D0007FD52B490027086940194608B219801A8D
:1027E000086128480068F6F715FA0022264BF6F72C
:1027F00067F9019100903E212846F6F735FF8019D0
:102800007941F6F715FA019B009AF6F7F1F8F6F719
:102810005BFA05461D4A0023F5F7DEFC06461B4918
:10282000F6F722FF1A49281A081A81B22204194819
:10283000324342600160206B0821884308432063D3
:10284000A069072109078843A061A169012081438C
:102850000143A1612062FCF7B5FD0F48104A0078E2
:10286000410041180D4808184178D1610D49807820
:10287000C8600D48077003B0F0BD00000080024042
:10288000A80200209000002000408F40710200004C
:10289000700200004080024010400020083D01010D
:1028A00040250240802502408000002000B50A46F5
:1028B00083B000210091019101466846F6F7A3FB21
:1028C0000199009803B000BD704770474368826863
:1028D00001699A60836842685A604A68824201D1FD
:1028E00082684A60002202610868401E0860086829
:1028F000704700000148006970470000A4470020AD
:10290000F8B51746204A06460024906B0725401C60
:1029100090631069814232D314206D1E1B496843B5
:1029200041182420604380190122FFF779F9041926
:10293000002DF1D12420144D6043801902226968D2
:10294000FFF76EF904192420604380190222A96858
:10295000FFF766F9041924206043801904220C490A
:10296000FFF75EF904192420604380190322094906
:10297000FFF756F90419002F01D00020386000F04D
:10298000DBFE2046F8BD0000A4470020D85C0020F4
:10299000A05D0020B45D00200146083100224160A6
:1029A000D243C16082600161002101607047002153
:1029B0000161704730B40C68621C02D002460832D4
:1029C00002E0026904E01A4653681D68A542FAD97C
:1029D00053684B6099608A60516008610168491CC6
:1029E000016030BC704742684A6093688B609368AE
:1029F0005960916008610168491C016070470000DE
:102A000072B604480168491C0160BFF34F8FBFF3E1
:102A10006F8F7047F847002005490868002804D0E8
:102A2000401E086000D162B6704772B6FEE7000033
:102A3000F847002000281CD070B504460D4D083C16
:102A40006068E968084201D172B6FEE72268002A90
:102A500001D072B6FEE78843606000F01BF9606841
:102A60006968401868602046FFF7B0F800F064FE1F
:102A700070BD7047E047002001200449000748600E
:102A8000BFF34F8FBFF36F8F7047000000ED00E082
:102A900010B500280FD009498A6B002A01D072B600
:102AA000FEE78A6B521C8A630021FFF701F800F0F1
:102AB00043FE002801D1FFF7DFFF10BDA44700202F
:102AC00002498A6A0260496941607047A447002050
:102AD000F0B585B00027054607702C4801690291C2
:102AE000006924214843FFF745F906004CD0002235
:102AF0000299FFF705FF03970290002841D9039838
:102B0000242148438019017B052911D20A007A4407
:102B1000127992189744020406080A00582408E023
:102B2000522406E0422404E0532402E0442400E05E
:102B3000002441682846F5F7E7FB2846F5F7B8FB7F
:102B40000F2804D220212954401C0F28FBD32F54D6
:102B50002D180398242148438019018C8268019222
:102B60000091036922460AA12846F8F79DFC2846F1
:102B7000F5F79EFB451903980299401C0390884283
:102B8000BDD33046FFF756FF05B0F0BDA447002087
:102B90000925630925750925750925750D0A0000A4
:102BA0000149012048627047A447002010B50C4637
:102BB000002809D0054909681831FFF7FBFE0121FB
:102BC0002046FEF775FF10BD72B6FEE7A447002051
:102BD00070B50B4604002FD0226D002A0ED0E16C98
:102BE000994200D21946E06A884225D0012A23D1B1
:102BF000124D2A68944203D172B6FEE772B6FEE720
:102C0000E162A269002A02DB0722511AA1611422A3
:102C10000B4E50436169801981420DD1201DFFF791
:102C200055FEE06AA969884200D9A8611421484389
:102C30008019211DFFF7D7FE70BD0000A4470020BA
:102C4000D85C002010B582B00D48002401902346C6
:102C500080220CA100940D4800F090FB012803D0C5
:102C6000401C0BD172B6FEE772B600210848C9437A
:102C700001630121C161446100F052F802B010BD4E
:102C8000D847002049444C4500000000791B010151
:102C9000A44700200248816B491C816370470000F3
:102CA000A4470020164B986B002802D001205862E0
:102CB0007047002058629869142102464A4311491E
:102CC0008A58002A0AD1002806D01422401E424306
:102CD0008A58002AF7D001E072B6FEE7142210B439
:102CE000424351184A680C46526808344A60A2426E
:102CF00001D152684A60D1681960986110BC704770
:102D0000A4470020D85C00200148406870470000BC
:102D1000E04700200148806870470000E04700203D
:102D200070B50F48016AFF22120411430162016A63
:102D30001202114301620B4C00252561A5610A486E
:102D40007D21C9000068F5F71DFA401E606107206B
:102D5000206106480560F5F7CBF9002070BD000042
:102D600000ED00E000E000E000400020F847002017
:102D700010B502460021012000F00CF8041E07D017
:102D80000021416001600B460A46C16000F05BF81B
:102D9000204610BDF8B517460E46050016D0002E89
:102DA00016D070435030FEF7E5FF04000CD02046EB
:102DB0005030002E0ED02060266420460121E563AD
:102DC00000F00AF84C2007552046F8BD72B6FEE721
:102DD0000020E7E72460EFE770B50D46040026D039
:102DE000FFF70EFE216CE06B4843216841186160DB
:102DF0000021A1632168A160E06B216C401E484363
:102E00002168224641180020C0434032E160107121
:102E1000507120461030002D0BD0FFF7BDFD20462D
:102E20002430FFF7B9FDFFF7F7FD012070BD72B642
:102E3000FEE721690029F6D000F04CFC0028F2D012
:102E4000FFF71AFEEFE7FFB5002783B0044600281E
:102E500003D00498002802D006E072B6FEE7206C8A
:102E6000002801D072B6FEE70698022804D1E06B74
:102E7000012801D072B6FEE700F03CFB002804D127
:102E80000598002801D072B6FEE72046254610308E
:102E900040350290FFF7B4FDA06BE16B884208D388
:102EA0000698022805D0059800284AD0002F4BD05C
:102EB0004EE0069E0499A56B0027226C002A11D0D3
:102EC000002E19D0E068F5F7CFF9E168206C091AF7
:102ED000E1602268914202D26168081AE060022E25
:102EE00017D019E02068002816D1606800F082FB36
:102EF0000746002060600FE0A068F5F7B5F9216C87
:102F0000A0684018A0606168884205D32068A0606E
:102F100002E0002D00D06D1E6D1CA563606A0028C4
:102F200006D02046243000F0D5FB002802D103E073
:102F3000002F01D0FFF7A0FDFFF76EFD012007B0C5
:102F4000F0BDFFF769FD20E06846FFF7B9FD0127F6
:102F5000FFF762FDFFF79EFEFFF752FD04202856A3
:102F6000401C00D1287105202856401C00D16871F2
:102F7000FFF752FD05A9684600F0CEF9002807D0FA
:102F80002046FEF7BDFE00F0D7FB002007B0F0BDE5
:102F9000FFF736FDA06BE16B884201D1012600E00E
:102FA0000026FFF739FD002E0ED005990298FFF795
:102FB000FDFD2046FEF7A4FE00F0BEFB002800D079
:102FC00068E7FFF759FD65E72046FEF799FE00F038
:102FD000B3FB5FE7FFB583B01E461746040003D07E
:102FE0000498002802D006E072B6FEE7206C0028A4
:102FF00001D072B6FEE7022E04D1E06B012801D0A9
:1030000072B6FEE7F5F788F80190A06BE16B884295
:1030100008D3022E06D000240198F5F781F8204647
:1030200007B0F0BD20464030052500904557324698
:1030300020460499FEF768FD681C04D000986D1CBA
:1030400045710124E8E7606A0028FAD02046243060
:1030500000F040FB0028F4D0002FF2D001203860AF
:10306000EFE7F7B5002784B00446002803D00598A1
:10307000002802D006E072B6FEE7206C002801D0DE
:1030800072B6FEE700F036FA002804D10698002850
:1030900001D072B6FEE72046254624304035029026
:1030A000FFF7AEFCA66B002E21D0226C059B002AF8
:1030B0000BD0E0688018E0606168884201D3206826
:1030C000E06001461846F5F7CFF8761EA663206942
:1030D000002807D02046103000F0FCFA002801D06C
:1030E000FFF7CAFCFFF798FC012007B0F0BD069877
:1030F000002802D0002F05D008E0FFF78DFC00204B
:1031000007B0F0BD6846FFF7DBFC0127FFF784FC42
:10311000FFF7C0FDFFF774FC04202856401C00D1C7
:10312000287105202856401C00D16871FFF774FCF7
:1031300006A9684600F0F0F8002811D02046FEF7F6
:10314000DFFD00F0F9FAFFF75BFCA06B002827D049
:103150000026FFF761FC002EA2D0002007B0F0BDD2
:10316000FFF74EFCA06B002812D00026FFF754FC9E
:10317000002E0FD006990298FFF718FD2046FEF7A3
:10318000BFFD00F0D9FA00288AD1FFF775FC87E768
:103190000126EBE72046FEF7B3FD00F0CDFA7FE70E
:1031A0000126D6E7F3B5002785B00446009700282E
:1031B00004D0206C002803D072B6FEE772B6FEE79A
:1031C00000F098F9002804D10698002801D072B6C2
:1031D000FEE720462546243040350190FFF710FCDD
:1031E000A06B002817D0401EA0632068002802D1E1
:1031F000FEF73AFE60602069002807D020461030B4
:1032000000F068FA002801D0FFF736FCFFF704FC55
:10321000012007B0F0BD0698002802D0002F0AD088
:103220000DE00098002801D072B6FEE7FFF7F4FB2E
:10323000002007B0F0BD02A8FFF742FC0127FFF70E
:10324000EBFBFFF727FDFFF7DBFB04202856401CB4
:1032500000D1287105202856401C00D16871FFF765
:10326000DBFB06A902A800F057F800281BD0204677
:10327000FEF746FD00F060FAFFF7C2FBA06B0028E6
:103280003ED00026FFF7C8FB002EA7D000980028EC
:103290003ED0FFF7B5FB606A002833D0206B0721D2
:1032A0000068091A2FE0FFF7ABFBA06B002808D0DD
:1032B0000026FFF7B1FB002E1CD02068002802D0AA
:1032C00009E00126F5E7FFF79BFB606800F0C6F90F
:1032D0000090FFF7A1FB06990198FFF767FC2046D5
:1032E000FEF70EFD00F028FA002800D076E7FFF781
:1032F000C3FB73E72046FEF703FD00F01DFA6DE700
:103300000126BFE700216068FFF762FCFFF784FB3E
:10331000002007B0F0BD0000F8B50D46040012D043
:10332000002D12D0FFF76CFB134E7269636828689A
:10333000D11A471C0BD02768B66AB74209D093420E
:1033400007D8012413E072B6FEE772B6FEE7002448
:103350000DE0884208D9401A28600748816A216038
:1033600040696060002402E0002001242860FFF72B
:1033700053FB2046F8BD0000A4470020FFB585B0F0
:1033800090000F9F0E9D0290FEF7F4FC06001ED0E9
:103390005C20FEF7EFFC040016D02663059901912E
:1033A0000899009130460299069EA5220391F4F7F0
:1033B0006DFF0399206B091F4018C008C0000290E0
:1033C000400708D072B6FEE73046FFF733FB002017
:1033D000C04309B0F0BD2118325C20310A75315C60
:1033E000002902D0401C1028F5D326460020403684
:1033F000F070072D00D30625E5620020E564206506
:10340000201DFFF7D4FA20461830FFF7D0FA2461C8
:103410000720411B6462A161002161653176009A39
:1034200001990298FEF72CFD2060002F00D03C602F
:103430002546FFF7E5FA284E3069401C30613068B8
:10344000264F002803D0F069002821D026E03560FF
:103450003069012822D1002414206043C019FFF7ED
:103460009BFA641C072CF7D31D48FFF795FA1D48FB
:10347000FFF792FA1C48FFF78FFA1C48FFF78CFA07
:103480001B48FFF789FA164870601430B06005E0F9
:103490003068E96AC06A884200D83560F06A401C2A
:1034A000F0626864E86AB169884200D9B0611421A9
:1034B0004843C019291DFFF796FAFFF7ADFAF069E6
:1034C000002806D03068E96AC06A884201D2FFF756
:1034D000D3FA012009B0F0BDA4470020D85C002039
:1034E000645D0020785D00208C5D0020A05D0020E0
:1034F000B45D00200648C169002904D0806B002813
:1035000003D0002070470120704702207047000060
:10351000A44700200148406970470000A4470020EC
:10352000F8B5324F0026B86B002808D0386A401C26
:103530003862786A002800D001263046F8BD7D69DF
:103540006D1C7D6115D178680068002801D072B6C5
:10355000FEE77868B9687960B860B86A401CB862FC
:1035600078680068002813D07868C068C068406830
:103570003863386B854211D37868006800280AD018
:103580007868C068C4686068854211D2386305E015
:103590000020C043ECE70020C043386338681421A2
:1035A000C06A4843124908580128C2D90126C0E719
:1035B000201DFFF78BF9A06A002803D020461830A1
:1035C000FFF784F9E06AB969884200D9B86114212B
:1035D000484307494018211DFFF705FAE06A39689A
:1035E000C96A8842C8D30126C6E70000A447002064
:1035F000D85C002070B500210446002828D0154D65
:103600002868844201D072B6FEE7206D002808D0F9
:10361000401E2065E36CE26A9A4219D0002802D06D
:1036200016E072B6FEE7201DFFF750F9E06C0721A7
:10363000E062081AA061E06AA969884200D9A8611D
:103640001421484304494018211DFFF7CCF90121FA
:10365000084670BDA4470020D85C002070B5044621
:103660000020002C2AD0194DE16A2A68D26A9142C2
:1036700025D2A069002804DB28680721C06A081A3F
:10368000A061E06A1422124E5043616980198142A0
:1036900010D1201DFFF71AF92868C06AE062A969F5
:1036A000884200D9A861142148438019211DFFF7E1
:1036B0009AF902E02868C06AE062012070BDE16CFE
:1036C0002A68D26A9142F8D370BD0000A447002056
:1036D000D85C002070B5C068C468002C0BD02046B0
:1036E00018300646FFF7F2F8104DA86B002804D0FA
:1036F00031460F480EE072B6FEE7201DFFF7E6F8F0
:10370000E06AA969884200D9A8611421484309499F
:103710004018211DFFF767F9E06A2968C96A8842E5
:1037200002D90120686270BD002070BDA44700204E
:103730008C5D0020D85C0020F8B52E4D0027A86BCA
:10374000002808D0FFF75CF9A86B401EA863A86B9F
:10375000002802D046E072B6FEE72869002841D072
:10376000254E306800282AD0F068C46820461830FA
:10377000FFF7ACF8201DFFF7A9F8E06AA9698842B5
:1037800000D9A861142148431C494018211DFFF7A6
:103790002AF9E06A2968C96A884201D3012068626F
:1037A00030680028E0D1002C09D0686829460068FC
:1037B00000281BD04868C068C068406808632C6A4D
:1037C000002C09D00126FFF7ABFE002800D06E6266
:1037D000641EF8D100202862686A002802D0012700
:1037E000FFF74AF9FFF718F93846F8BD0020C04343
:1037F000E4E70000A44700208C5D0020D85C002096
:1038000040BA7047C0BA70470138FDD17047000018
:10381000F7B50325AD06286A82B016460C46400867
:1038200040002862286A022108432862286A80072B
:10383000FCD46620686001272F61A86AC005FCD50A
:10384000992068602F61A86AC005FCD5FF209130DF
:10385000FFF7DAFFFF230133AB626846EF603521E3
:1038600069602F61A96AC905FCD5AB62A969EF60DF
:10387000C9B205226A602F61AA6AD205FCD5AB6283
:10388000AA690902D2B211430180C80702D00320FD
:1038900005B0F0BDAB626869FF21083188436861FB
:1038A0006869C91E08436861029800024830686070
:1038B0000820A860EE602F61A86AC005FCD5FF2033
:1038C0000130A8620023F61CB0080ED0B2081148DF
:1038D000006899006054060A09194E70060C000E23
:1038E0008E705B1CC8709A42F1D8FF200130A8622C
:1038F0006869FF21083188436861686938436861F5
:10390000286A800880002862286A384328620020DC
:1039100005B0F0BD8000000C032080064169FF2245
:10392000083291434161426901210A434261026ABE
:10393000920892000262026A0A4302627047000023
:10394000002003218906096A4908490003229206DA
:1039500011621146096A0222114303229206116282
:1039600000BF03218906096A022211400229F8D00A
:10397000D1010322920691620321D1609F215160FF
:103980000121116100BF03218906896AFF220132EA
:1039900011409142F7D10322920691621146886943
:1039A0004969FF2208329143032292065161114670
:1039B0004969012211430322920651611146096AA5
:1039C0008908890011621146096A01221143032204
:1039D0009206116270470000000001020000000022
:1039E000010203040138FDD170470000F0B4032444
:1039F000A406236A5B085B002362236A02252B432B
:103A00002362236A9B07FCD4FF230133A362656909
:103A1000DE1DB543656165691E1D354365610002A4
:103A20006B3060600820A060E26001262661A06A19
:103A3000C005FCD5A3620023D21C90080ED09508C7
:103A40000F4800689A008854070A52185770070CEC
:103A5000000E97705B1CD0709D42F1D86069FF2109
:103A6000083188436061606930436061206A800882
:103A700080002062206A30432062F0BC0020704742
:103A80008000000CF8B5064601200025C0048642DF
:103A900001D90520F8BD0324A406206A400840008F
:103AA0002062206A022108432062206A8007FCD439
:103AB000FF270137A76200F0BBF8002801D00325DB
:103AC00015E00620606001212161A06AC005FCD5D7
:103AD000A7623002203060602161A06AC005FCD579
:103AE000A7620C4800F0C8F8002800D102256069E0
:103AF000FF210831884360616069012108436061EA
:103B0000206A800880002062206A084320622846DC
:103B1000F8BD0000E6960100F7B506460120C00496
:103B200082B01546864202D9052005B0F0BD0320BB
:103B30008006016A490849000162016A02221143B4
:103B40000162016A8907FCD4FF2101318162F2B26E
:103B50008C1AA54200D8ACB20398009000F068F827
:103B6000002840D106214806416001210161816A97
:103B7000C905FCD5FF21013103208006816241691E
:103B8000FF2208329143416141690422114341619E
:103B9000310232314160C4600022002C16D90098F5
:103BA00087183B78F87819467B7800061B02194382
:103BB000BB781B04194301430802F978000A09067F
:103BC000084319490860121DA242E8D301210320CD
:103BD00080060161816AC905FCD5FF21013181623E
:103BE000124800F049F8A54209D003983619001987
:103BF0002D1BFF2401340390A542ADD8ABE7032071
:103C000080064169FF2208329143416141690122E6
:103C100011434161016A890889000162016A114307
:103C20000162002005B0F0BD8000000C1A06000003
:103C300038B40125032080066A46C56035214160FD
:103C40000561816AC905FCD5FF240134846281695C
:103C5000C560CBB2052141600561816AC905FCD50B
:103C6000846280691902C0B2014388B21180C00722
:103C700000D0012038BC7047F8B400210125032290
:103C800092066B46D560352454601561946AE4054C
:103C9000FCD5FF27013797629469D560E4B2052609
:103CA00056601561966AF605FCD5976296692402FE
:103CB000F6B234431C80E30722D0814202D9F8BC1B
:103CC00000207047032292066B46D560352454606D
:103CD0001561491C946AE405FCD597629469D56026
:103CE000E4B2052656601561966AF605FCD5976222
:103CF00092692402D2B21443A2B21C80D207DCD152
:103D0000F8BC0120704700000017130017100017BF
:103D10000E001709001704001700001718011714E8
:103D2000011715011719000000280002000000000B
:103D30000328000200000000292A00020080800001
:103D40000328000200000000242A000200808000F6
:103D50000328000200000000252A000200808000E5
:103D60000328000200000000272A000200808000D3
:103D70000328000200000000262A000200808000C4
:103D80000328000200000000282A000200808000B2
:103D90000328000200000000232A0002008008001F
:103DA00003280002000000002A2A00020080080008
:103DB0000328000200000000502A000200800700D3
:103DC000D9D9000167D9000165D9000163D9000183
:103DD0000014000081DA0001130C0000BDEC0001AA
:103DE000031400003DDB0001A72001012120010197
:103DF000D51F0101891F0101130C000081ED000195
:103E0000150C000061EE0001170C000099EB000199
:103E1000000C0000D9EB0001064700004F23010110
:103E200003470000F5230101084700009522010126
:103E30000E470000E11E010105470000A925010110
:103E4000FFFF000011CC0001130E0000D9DE0001BD
:103E5000150E0000E9DD0001170E000059E3000116
:103E6000190E000031E30001403E01010500000091
:103E7000F7B586B0002002905C48154604695C489E
:103E80000E46824201D9054602E0002D00D10125EF
:103E9000002C08D0A1880698814204D1E088B04265
:103EA00001D10120029053480390844606980104F2
:103EB00031430020002C1CD00A0CA7888BB29742FB
:103EC00007D1E7889F4204D1002807D0216801600C
:103ED00007E020462468002CEFD10AE06146226802
:103EE0000A602168002902D00020206001E06146BC
:103EF0004860002C07D10221102000F095F80699A7
:103F000081800446C6802801052100F077F8074625
:103F10007D200E464643EFF31085012080F3108884
:103F2000684600F087F885F3108800980490C0195F
:103F30000501019927202D098E190001059186425E
:103F400003D96D1C2D012D09361AE660A560039872
:103F5000294F86460020844670460068002813D00A
:103F6000A268E1680091C36881680193531A1B013C
:103F70001B09BB420AD2914203D1019A0099914296
:103F800004D984460068E9E77246546020606046C0
:103F9000002801D0046001E071460C6013480299CA
:103FA0000069002901D1A04203D1C168806800F0F6
:103FB00047F8EFF31084012080F3108802A800F086
:103FC00039F884F31088039902980191291A09019C
:103FD00009090090B94204D2A84205D1019886424D
:103FE00002D8032000F032F809B0F0BDC80100206B
:103FF000FFFF7F02D8010020FFFFFF0730B50B460F
:10400000014600202022012409E00D46D5409D42B2
:1040100005D31D469540491B254695404019154638
:10402000521E002DF1DC30BD03B40148019001BDEA
:104030002D7A010003B40148019001BD5DB6020074
:1040400003B40148019001BD9DB6020003B40148CC
:10405000019001BDAD78010030B4C3688268886802
:10406000084D141A2401C9682409AC4203D29042B5
:1040700004D18B4202D830BC0120704730BC0020F4
:1040800070470000FFFFFF070A0C838889B2934244
:1040900004D1C088884201D10120704700207047B8
:1040A00070B4054600680022002810D00B0C8688EA
:1040B0008CB29E4207D1C688A64204D10168002A6C
:1040C00007D0116006E0024600680028EFD170BCFE
:1040D000704729600168002903D00021016070BC8D
:1040E00070476A6070BC7047F0B5104F0268864632
:1040F0000025002A10D0C8688C6893688446E01AAE
:1041000000010009D668B84208D2A34201D1B445E3
:1041100004D915461268ECE7704641600A60002D2C
:1041200001D02960F0BD70460160F0BDFFFFFF07C0
:1041300070B584B004460E46EFF31085012080F37D
:10414000108802A8FFF776FF85F31088029803997C
:10415000024600900191A01A000107490009884217
:1041600004D2A24205D10198864202D8012004B0AF
:1041700070BD002004B070BDFFFFFF0730B583B0F5
:104180000446EFF31085012080F310886846FFF79E
:1041900051FF85F31088019900986160206003B099
:1041A00030BD0000002800020000000003280002CB
:1041B00000000000002A000A0080200003280002FE
:1041C00000000000012A0002008002000328000213
:1041D00000000000042A00020080080003280002FA
:1041E00000000000A62A000200800100032800024F
:1041F00000000000C92A000200800100002800021F
:10420000000000000328000200000000052A002032
:10421000008004000229000A0000020003280002B6
:1042200000000000292B000A008010000328000273
:10423000000000002A2B000200801000FFFF000099
:1042400011C70001A40D0000FDE50001A50D00004F
:1042500031E600011A0D000049EB0001150D0000C8
:1042600091E60001000D0000BDE600011C0D0000FC
:104270007FEB0001A70D00009DEA0001A80D0000E2
:104280008BEB0001020C000071EC0001000C00003F
:1042900049EC0001010E000075E100010F0E000065
:1042A00031E50001110E000095E500012C0E000023
:1042B00015E50001030E0000CDE200010A0E00002A
:1042C00089E40001300E000009E500010C0E000039
:1042D000BDE50001000E0000E1E00001090E000054
:1042E00009E10001010F000039C90001020F0000BF
:1042F000D9C50001030F00001DC90001040F000013
:104300006D0401013C420101364700200100190003
:1043100002140000B9DB000110430101010000009C
:104320002C4401010300000001102EC78A0E739077
:10433000E111C20860270000002800000000000012
:104340000000000000000000000200000000032840
:104350000000000000000000000000000000000A53
:104360000000000001002EC78A0E7390E111C20800
:1043700060270000000400C00002012900000000C6
:1043800000000000000000000000000A008014008F
:1043900003280000000000000000000000000000F2
:1043A000000A0000000002002EC78A0E7390E1117F
:1043B000C20860270000001000C0000202290000AF
:1043C000000000000000000000000000000A008063
:1043D000140003280000000000000000000000009E
:1043E0000000000A0000000003002EC78A0E739030
:1043F000E111C20860270000000A00C00002032883
:104400000000000000000000000000000000000AA2
:104410000000000004002EC78A0E7390E111C2084C
:1044200060270000000200C00002000004470000F6
:104430002D2501010A47000015240101074700004E
:1044400045230101C04701018C470101A1A60001DC
:10445000684701015047010151AA0001704701015D
:104460007446010179A8000184470101B0450101AA
:1044700099A400011C4701011846010121A4000173
:10448000E0460101B046010175A70001F8470101AE
:10449000EC450101E99B0001084801015848010170
:1044A000B19C0001C8470101244701015D9800014A
:1044B000104801017845010191980001004801016F
:1044C0005446010145A80001504801011848010166
:1044D00011A6000148480101E44601010DAA0001AE
:1044E00078470101D047010161A9000101020304DD
:1044F000050600404040404040404040414141416D
:1045000041404040404040404040404040404040AA
:1045100040404005020202020202020202020202BE
:10452000020202202020202020202020200202023F
:1045300002020202909090909090101010101010B3
:104540001010101010101010101010101010020287
:1045500002020202888888888888080808080808F3
:1045600008080808080808080808080808080202D7
:1045700002024000F34401016273736574203C66DB
:1045800069656C643E203C76616C3E3A20777269C6
:10459000746520626F6F7473657474696E672066EA
:1045A00069656C6420286361726566756C212900F9
:1045B00073686F772064657669636520696E666FDE
:1045C000202874656D702F7664642F66616E2C20D0
:1045D00073616D6520617320424C4520494E464F02
:1045E0005F515545525920616C6C290061707067AC
:1045F0006574205B6A736F6E5D3A2073686F772015
:1046000061707020706172616D7320286C65642F19
:1046100070776D2900000000626C656C6F67205B2D
:104620006F6E7C6F66665D3A20424C452074726105
:1046300066666963206C6F6720286576656E7473A3
:10464000202B206672616D65206865782064756D29
:104650007029000072657365743A2073797374650C
:104660006D20726573657420287265626F6F74299E
:104670000000000073686F77204672656552544FE2
:10468000532072756E74696D6520696E666F20289F
:10469000757074696D652F7461736B732F686561D4
:1046A000702F7461736B206C6973742900000000B3
:1046B0006C6564203C317C323E203C6F6E7C6F66C2
:1046C000667C746F67676C653E3A20636F6E7472C8
:1046D0006F6C20626F617264204C454400000000E2
:1046E0006C656400756172747273743A2072652D22
:1046F000696E697420555341525431202831313547
:1047000032303020384E31292C20666C7573682089
:10471000727820717565756500000000626C656CCB
:104720006F670000627364756D703A2073686F770D
:1047300020626F6F7473657474696E67207265634D
:104740006F7264202B2063726320636865636B0063
:1047500073686F77206669726D7761726520766520
:104760007273696F6E00000076657273696F6E0018
:10477000737973696E666F0075617274696E666FC6
:1047800000000000646576696E666F0068656C7095
:10479000205B636D645D3A206C69737420636F6D98
:1047A0006D616E6473202F2073686F77206F6E6564
:1047B00020636F6D6D616E6427732068656C700097
:1047C00068656C7000000000627364756D700000B5
:1047D00075617274696E666F3A2073686F772055E1
:1047E00053415254312070696E732F626175642F8A
:1047F000666F726D617400006170706765740000AF
:1048000072657365740000006170707365740000F8
:104810006273736574000000666163746F72793A45
:1048200020726573746F726520706172616D7320A0
:10483000746F2064656661756C747320616E6420AA
:104840007265626F6F7400007561727472737400C8
:10485000666163746F727900617070736574203C77
:104860006C65647C70776D3E203C76616C3E207C8C
:1048700020617070736574206A736F6E207B226C88
:104880006564223A3530307D000000007573616741
:10489000653A20617070736574203C6C65647C704F
:1048A000776D3E203C76616C3E207C206170707399
:1048B0006574206A736F6E207B226C6564223A35C2
:1048C00030302C2270776D223A35307D0D0A000091
:1048D0002020202020202020206231616464727C0E
:1048E0006232616464727C623173697A657C6232BF
:1048F00073697A657C62316372637C62326372636E
:104900007C62317665727C6232766572203C6865C5
:10491000787C6465633E0D0A000000003C4901019B
:10492000004000200C08000030950001504F0101AC
:104930000C480020BC6F0000F02A0000A006009088
:10494000D00300011005A00000FF01D20001000605
:1049500051C20200200001302B11D80D49086849CE
:104960006813F008FB0498EFF78EFF0446C18880B7
:1049700088FF22FFF79DFD2046FFF73AFCB3E705CD
:10498000B0F0BD98100707D8010020C804202930D6
:10499000D70200004B1847FBFD0646052030707516
:1049A000800099B181301D3946E5F773FD3046F935
:1049B000F70EFF0E22294642200445FD0740301124
:1049C0002E0CD0534B052203212846FDF733FE124F
:1049D0001E40274B75002D05D0398F002902D000CD
:1049E00099897900E000211176FAF74BF8044D28F7
:1049F00059F9F7FBFE002028518010060004002022
:104A00000777107838B5049C0094014CA04738BD56
:104A10005143F84A26468F1839462036FD6D707D81
:104A200080311191C97FA0370E9122463978153215
:104A30000F92F14A109203292BD0002873D0F17DF8
:104A40000F980CF00DF800286FD06888694608832D
:104A5000F0B597B008780C460F90002014900F988E
:104A600048214843FE4922464018064680361090A9
:104A7000F17F0091C56DA0301690014E100A2746B7
:104A800012922037F74A1552146C2AD061783C29CB
:104A900049D0432947D0787D00287DD0F97D1298F0
:104AA00000F0FCF9002878D0698868468184687A2B
:104AB000297A000409020843E97908430690A97A93
:104AC00008A84172E97A8172297BC17229460D31A9
:104AD0000E380E9100F02FFAA878400733D5002148
:104AE00032E0907E012806D0507E401E0006000E67
:104AF000507603D006143004DB480106141200F08F
:104B0000D2F9169A01211170A978D448C9075C36E8
:104B100090264823594308180022A0300270FF2035
:104B2000F07752E001220270A878CC49C0074CD03F
:104B30000098482358434020101442E0E97C08A81C
:104B40000173297D4173697D8173A97DC108100DB1
:104B50000174297E4174697E8174B189BC102281FF
:104B6000F189C181318A0182109940318A8F828313
:104B7000C98F0184B188C183F18841840021C18437
:104B800042241472B848817808A8C17401E04DE14C
:104B90001BE002260675C821CC140C02D4E87A80EA
:104BA0000705D5297B0E14300A7EF908A90875037C
:104BB000A90F0C1412002801D11698067060783CD9
:104BC0002870D030E1628A143D0A82A2884A82A20B
:104BD000790A75E2794A75207A8875E07EC875A0F1
:104BE0008B0883E08B4883208C8883608CC883216A
:104BF00046243108A800F0A4F9787A08A94871B8C9
:104C00007A8871A08DC8140585206B0BC210050C25
:104C100090012018103F75387D0875B87D8875A8FB
:104C200078C006C017401CC8758E486946028A0ABB
:104C300087428A4A87827D08A90A77C27D4A77021D
:104C40007E8A77428B10A90A80828B4A80807F08F7
:104C50007104A900A4380432F9000A14487C4940C0
:104C60001803907C30129900F05DF90398F97D806B
:104C700030817003990922A0310A700121C17003AB
:104C80009800218166E18B490041660521C16601DA
:104C90006715996030C97E002904D072498161018D
:104CA0002102E02ABA480981618175009981822434
:104CB000400DF6F8022802D2012100F003F912207B
:104CC0001B05F906280CD20A215F4A41438918FFC7
:104CD000318131497F890703D5FA7D7C23FCF89621
:104CE0001005FFF81699E035C41A01AE181809200E
:104CF00000F0FBF821460F31059100284ED020230B
:104D00003E22002156241C06F6F806460A96031792
:104D100014986C1ED03A04200EE03C2070700120E4
:104D20003071009870801620052CD0B01D5A2407D1
:104D3000F2F8F87D7071AC201306D5214630460993
:104D4000310C3000F0E7F803E030460A12DD202590
:104D5000C8100630461230053032DA1A12121A1410
:104D600006D0F8E08B309A16709A2813B083B87A80
:104D7000B077304600F0BFF83AE0287B7071DC2055
:104D800007B01D00F0C2F8163006B4F83DE0149EDE
:104D90001A2EC23008A7F801210646019E120D9E68
:104DA000300470703198200BF87D820709D571713D
:104DB000B01D6A3004A5F80AB6400B30461DE0C0AD
:104DC00007C00F7071B2129978100BB081208CF06F
:104DD00081608C308278227462300483F80660121D
:104DE0001660302477F81421017000994180B97D54
:104DF000017100F075F81598807E022826D1607840
:104E00001499084322D0082C120B2C100461F812BC
:104E10002C1C0C61784170297881700FE04064048B
:104E20001C06C00600200A6E0512390412400C1D33
:104E300088031C0820B1A201000411A005100799E5
:104E40008180397E81563C064AF8002017180510EB
:104E50000640BA7047C004600D03B40148019001D8
:104E6000BD919B02000C83E1980C837D9F0C700424
:104E700049FA010C8309D30C836D5B24933D994857
:104E80008290488355073083D59C3083397B181036
:104E900027796D0100002101804180818070470ADF
:104EA0007802704B7843708A788270CA78C2700B2F
:104EB0007903714A7942711A20046802600E0F3436
:104EC000704740063414497B41700570F1F7F3FCDC
:104ED0002068F1F7A4FB256003141B2400761C094D
:104EE00080024080C10240062B066419F8B54E7856
:104EF0004821F0B248432349214D41180C46AA7E6F
:104F0000A0340027282C22EDC3020010B5074CE086
:104F100069000408D5FFF7F3FF0548007800280270
:104F2000D10120C0032062100006115012C6580F94
:104F30004EF4010607CD7007100699B5000135043F
:104F400000065529260101000112AA01E15C0000BA
:00000001FF
